:106FC0000000090200000301FA0400EF0500030AB3
:106FD0000A5A0B001E0C00FA0D00030E00040F01EC
:106FE00064100096120132130AFA14020217010A01
:106FF0001801EF1905321A010A1B01EF1C05321F97
:10700000FFFF20FFFF23011E2400642A00FA2B004B
:10701000FA2C50782D003D2E004630006432507816
:107020003300003432FA35016436016437015038D8
:107030000A643A00033B00043C00643E003C3F000D
:107040000140FFFF411450420A5A430AC844053226
:107050004500B44600FA4900024B00014C00FA50CA
:107060000808510596520A32530B46540A965705A2
:1070700046590A465A32FA5B010A5C0A325E000A35
:107080005F00646200FE64011167FFFF680101692F
:1070900001016A05966B00006C32966D0004730066
:1070A000007400007801327901327E00647FFFFFB6
:1070B00080FFFF8100008400648800028A00019D37
:1070C0000A969E00019FFFFFA0FFFFA2000AA3FFF8
:1070D000FFA4FFFFA5FFFFA6FFFFA7FFFFA8FFFF7D
:1070E000A9FFFF0101241502022F003C4701484877
:1070F00002035602024EFFFF58000261FFFF6600C6
:10710000028500AF8600018700FA8901079900080F
:10711000A100FAFAFAFA0101241502022F1E3C47D7
:1071200001484802035602024EFFFF58000261FF69
:10713000FF6600028500AF8600018700FA8901071B
:10714000990000A10000FAFAFA0065006F007900CA
:1071500083008D009700A100AC00B600C000CA00FB
:10716000D400DE00E800F200580060006800700003
:1071700078008000880090009800A000A800B0006F
:10718000B800C100C800D000D800DF00E600EE0063
:10719000F600410047004D00530059005F006500B4
:1071A0006C00710077007D00830089008F009500DE
:1071B0009B00A200A700AC00B200B900C000C5004F
:0D71C000CA00D200D500DD00E100E700EFBD
:103CD80085F97485FA757E017F00E5751272DFE556
:103CE800742FFF50010E8E5A8F5B90001CE0FCA3CE
:103CF800E0FDEF2DFDEE3CFC8C5C8D5D90003CE022
:103D0800FAA3E0FBED2BFBEC3AFA8A5C8B5D22759B
:103D1800A71085F97485FA757E017F00E575127222
:103D2800DFE5742FFF50010E8E5A8F5B9000F7E08D
:103D3800B40210AC2DAD2EEF2DFDEE3CFC8C5C8D4D
:103D48005D8016AE5AAF5B90001CE0FCA3E0FDEF6F
:103D58002DFDEE3CFC8C5C8D5DAE5CAF5D90003C57
:103D6800E0FCA3E0FDEF2DFDEE3CFC8C5C8D5D22BC
:103D7800E55DF5FBE55CF5FCD29322E55DF5E9E54B
:103D88005CF5EAD29422E55DF5EBE55CF5ECD291C1
:103D980022E55DF5EDE55CF5EED292229000D9E0E2
:103DA800C394045003123D17E55DF5FBE55CF5FC93
:103DB800D287229000D9E0C394045003123D17E53E
:103DC8005DF5E9E55CF5EAD290229000D9E0C3946C
:103DD800045003123D17E55DF5EBE55CF5ECE5B540
:103DE8004410F5B5229000D9E0C394045003123D65
:103DF80017E55DF5EDE55CF5EEE5B54420F5B52292
:103E080075E700A203B34008E5B54480F5B5800620
:103E1800E5B5547FF5B575E71022E50C906BB2F85F
:103E2800282873023EBF75E700A239B34008E5B5FC
:103E38004408F5B58006E5B554F7F5B575E7108083
:103E48007675E700A239B34008E5B54440F5B5807A
:103E580006E5B554BFF5B575E710805B75E700A2B8
:103E680039B34008E5B54480F5B58006E5B5547F1B
:103E7800F5B575E7108040A2399287803AA2399249
:103E880090803475E700A239B34008E5B54410F5D1
:103E9800B58006E5B554EFF5B575E710801975E7F7
:103EA80000A239B34008E5B54420F5B58006E5B56C
:073EB80054DFF5B575E710BA
:106BB200023E2B023E2E023E49023E64023E7F020C
:086BC2003E85023E8B023EA657
:103EBF00227433900168F07436900169F0742D907C
:103ECF00016AF0743190016BF0742D90016CF074F5
:103EDF003190016DF0742090016EF0744E90016F6F
:103EEF00F07469900170F07473900171F0746190C7
:103EFF000172F0746E900173F07420900174F0747D
:103F0F0056900175F07438900176F02290089FE07A
:103F1F00FEA3E0FF7423D39F74019E400C906FC0EB
:103F2F00120048E493F599802E90F802E493B405BB
:103F3F001490089FE0FEA3E0FF906FF3120048E497
:103F4F0093F599801290089FE0FEA3E0FF906FC059
:103F5F00120048E493F59990089F1272ED90089F14
:103F6F00E0FEA3E0FFEFB45607EEB40103754E0079
:103F7F0022AE5AAF5B740A8E048F05FF1272CF8C7C
:103F8F005C8D5DAE5AAF5B740A8E048F05FF1272A3
:103F9F00FA8C5A8D5BE55B455A6013740AC3955BC7
:103FAF00FFE4955AFE8E5A8F5B785C127332E5747C
:103FBF00A85CB80015D3955D4010E574C3955DFFFF
:103FCF00E4955CFE8E5C8F5D8010E5742424C395B0
:103FDF005DFFE4955CFE8E5C8F5DAE5CAF5D741231
:103FEF006F4E600674246F4E700A785C12733A75C8
:103FFF0074018003757400229000A5E0B40104C21F
:10400F00078002D2079000A6E0B40104C208800224
:10401F00D2089000E3E075F0E1A4FFAEF0740A8ED1
:10402F00048F05FF1272CF900893ECF0A3EDF09080
:10403F0000E3E075F02BA4FFAEF0900018EEF0A3B4
:10404F00EFF07E017F009000A1E01272DF9000E49C
:10405F00E08E048F05FF1272CF740AFF1272CF8D9C
:10406F00619000EDE075F0E1A4FFAEF0740A8E04EC
:10407F008F05FF1272CF900897ECF0A3EDF0900030
:10408F00EFE060139000EFE0F5F0741684FF7E0010
:10409F00EF9008F5F0800674649008F5F09000E555
:1040AF00E0900082F0900131E090008CF0900133AD
:1040BF00E0FE9000E1E08E0088F0A4FFAEF0EF90FC
:1040CF0008FEF090010CE075F013A4FDACF0900029
:1040DF003CECF0A3EDF0A225B3401690017DE0700B
:1040EF000C90017EE0700690017FE060028002C2BA
:1040FF002590017DE0B4300F90017EE0B447089029
:10410F00017FE0643B60028004D2268002C22674E5
:10411F00E3900081F09000CEE0B40B0874E39000C0
:10412F0081F0805A9000CEE0B419129000E4E09034
:10413F00713412008CE493900081F080419000CE96
:10414F00E0B41E129000E4E090715212008CE493E0
:10415F00900081F080289000CEE0B428129000E407
:10416F00E090717C12008CE493900081F0800F90AE
:10417F0000CEE0B446089000C5E0900081F09000BA
:10418F009EE0FE9008FFE06E601B7599E612019CA1
:10419F0074AB90005BF012069A7464F50975080011
:1041AF001205E480FE900096E0700674009000CB3C
:1041BF00F0900086E0FE9000CBE0B5063F900088BF
:1041CF00E0FE9000E9E0B50633900087E0FE900036
:1041DF00F7E0B5062790008AE0FE90009EE0B50656
:1041EF001B900089E0FE9000D9E0B5060F90008B80
:1041FF00E0FE900117E06E70030244159000D9E0C5
:10420F00D3940250069000F7E06008740390011AEF
:10421F00F08006740790011AF09000D9E0D3940251
:10422F0040089000F7E0640260028006740090007E
:10423F00F7F090009EE0B40106740090009EF0909D
:10424F00009EE0B4020674009000E9F090009EE03A
:10425F00B4030674009000F6F0900117E060147438
:10426F002990078FF074009006D7F074009006D84D
:10427F00F0800C740090078FF074299006D7F0909F
:10428F0000E9E0D39401402774009000B3F0741B51
:10429F0090011CF074009006DBF074009006DCF0C7
:1042AF009000CBE0B4020674019000CBF080339005
:1042BF0000CBE0B4021A741B9000B3F074009001AD
:1042CF001CF074009006DBF074009006DCF0801296
:1042DF0074009000B3F0740090011CF0741B9006F2
:1042EF00DBF09000F7E0B401089000D9E0640360C0
:1042FF00028026741C90011DF074009000B2F074BF
:10430F00009006DFF074009006E0F09000CBE060C4
:10431F000674009000CBF080329000CBE0601A74EE
:10432F001C9000B2F0740090011DF074009006DF35
:10433F00F074009006E0F08012740090011DF0748C
:10434F00009000B2F0741C9006DFF09000D9E0B43A
:10435F0002069000F7E06002803274059006E3F0E9
:10436F0074069006E7F074079006EBF07408900659
:10437F00EFF0740090078BF0740090078CF07400CE
:10438F0090078DF0740090078EF0804874009006AF
:10439F00E3F074009006E4F074009006E7F0740008
:1043AF009006E8F074009006EBF074009006ECF0C5
:1043BF0074009006EFF074009006F0F0740590070B
:1043CF008BF0740690078CF0740790078DF07408CB
:1043DF0090078EF0D2249000CBE0900086F09000F2
:1043EF00F7E0900087F09000E9E0900088F09000EF
:1043FF00D9E0900089F090009EE090008AF0900143
:10440F0017E090008BF0900101E0B40117900028A5
:10441F00740FF0A374FFF090002AE4F0A3F074027D
:10442F00900101F0900101E0B4034190002AE0FEF9
:10443F00A3E0FF900028E0FCA3E0FD12732A7410A4
:10444F001272DF7408120039EF900100F0EF70065E
:10445F0074FF900100F07400900101F0900029E0CA
:10446F009000B7F0900028E09000B8F0900092E034
:10447F0090008FF0900091E090008EF09000C0E0DF
:10448F00C3941E50569000C0E0F404241E90009078
:10449F00F0900090E075F00A84FF7E008F7490001A
:1044AF0090E075F00A84ADF07C008D7590008EE081
:1044BF00D39575400D90008EE0C3957590008EF0EA
:1044CF00800F90008EE0240AC3957590008EF00542
:1044DF007490008FE0257490008FF090008FE09023
:1044EF00004EF090004EE0D39424400B90004EE02D
:1044FF00C3942490004EF090004EE0240990004F9A
:10450F00F090004EE02412900050F090004EE02406
:10451F001B900051F090004FE0D39424400B90007B
:10452F004FE0C3942490004FF0900050E0D39424B8
:10453F00400B900050E0C39424900050F090005135
:10454F00E0D39424400B900051E0C3942490005189
:10455F00F0900056E4F090004EE064126007900077
:10456F004EE0B4241B9000567401F090004EE0B45E
:10457F001208741190004EF0800690004E7401F0F6
:10458F00900057E4F090004FE06412600790004FE6
:10459F00E0B4241B9000577401F090004FE0B41268
:1045AF0008741190004FF0800690004F7401F09046
:1045BF000058E4F0900050E064126007900050E063
:1045CF00B4241B9000587401F0900050E0B412080E
:1045DF007411900050F080069000507401F090001C
:1045EF0059E4F0900051E064126007900051E0B47C
:1045FF00241B9000597401F0900051E0B41208741C
:10460F0011900051F080069000517401F0900092CB
:10461F00E0FE9000F5E02E90005CF090005CE0640E
:10462F0012600790005CE0B4240690005CE004F098
:10463F0090005CE0D39424400B90005CE0C3942482
:10464F0090005CF090005CE0D39412400D90005C01
:10465F00E0C3941290005DF0800A90005CE0241299
:10466F0090005DF0755E129000D8E0900052F090CF
:10467F000052E075F00984AFF07E00EF4E700690A7
:10468F000052E004F0900052E0B4250690005274FE
:10469F0001F0900052E0D39424400F900052E0C3F9
:1046AF009424900052F0D21F8002C21F900052E05B
:1046BF002409900053F0900052E02412900054F01F
:1046CF00900052E0241B900055F0900053E0D394DB
:1046DF0024400B900053E0C39424900053F09000BB
:1046EF0054E0D39424400B900054E0C394249000E2
:1046FF0054F0900055E0D39424400B900055E0C344
:10470F009424900055F012019C22C293C294C2913E
:10471F00C292C287C290E5B554EFF5B5E5B554DF47
:10472F00F5B5C296C295C2A0C297C2A2C2A1E5B505
:10473F0054BFF5B5E5B5547FF5B5E5B554FBF5B503
:10474F00C209755F469000DBE07005756E0280034D
:10475F00756E0375550075540090001074FFF0A32B
:10476F0074DCF0C210C212C214C21674C890003E9C
:10477F00F074C8900042F074C8900046F074C8906E
:10478F00004AF0755300755200C204754700E5707A
:10479F00B4130375700075640090001EE4F0A3F06D
:1047AF00757110C20CC20DC20EC20FC20375570035
:1047BF00755600900012E4F0A3F0900014E4F0A3FB
:1047CF00F0C22975590075580090009DE075F032C0
:1047DF00A4FFAEF0900026EEF0A3EFF090008DE472
:1047EF00F09008FBE4F0C227D21CC21BD21DC21EE0
:1047FF00C21FC220900016E4F0A3F022755B007573
:10480F005A00AE5AAF5B7422C39F74019E500302CD
:10481F0048FF906FC0120048E493645F6023906F6D
:10482F00C0120048E493647E6017906FC012004876
:10483F00E4936481600B906FC0120048E493B484DA
:10484F00030248DFAE5AAF5B906FC0120048E4938B
:10485F009000911273100FBF00010EE0FC906FC01B
:10486F00120048ECFEE493FFEEC39F5026AE5AAF02
:10487F005B0FBF00010E906FC0120048AE5AAF5BC6
:10488F00E493FC906FC0120048E493900091127370
:10489F0010ECF0AE5AAF5B906FC0120048E49390EB
:1048AF000091127310E0FC906FC2120048ECFCE410
:1048BF0093FDECD39D4019906FC2120048E493FC16
:1048CF00906FC0120048E493900091127310ECF0B7
:1048DF00AE5AAF5B74022FFF50010E8E5A8F5B786A
:1048EF005B740126F6500418E436F64003024811B3
:1048FF0022755B00755A00AE5AAF5B7432BE00036F
:10490F009F50030249CD9070E3120048E49390004A
:10491F00911273100FBF00010EE0FC9070E31200B4
:10492F0048ECFEE493FFEEC39F5026AE5AAF5B0FE9
:10493F00BF00010E9070E3120048AE5AAF5BE493D4
:10494F00FC9070E3120048E493900091127310EC06
:10495F00F0AE5AAF5B9070E3120048E49390009171
:10496F00127310E0FC9070E5120048ECFCE493FD2C
:10497F00ECD39D40199070E5120048E493FC9070C1
:10498F00E3120048E493900091127310ECF0AE5ACA
:10499F00AF5B742D6F4E7006755B33755A00AE5A50
:1049AF00AF5B74022FFF50010E8E5A8F5B785B74D2
:1049BF000126F6500418E436F64003024906227524
:1049CF005B00755A00AE5AAF5B7432BE00039F5046
:1049DF0003024A9B907116120048E49390009112C3
:1049EF0073100FBF00010EE0FC907116120048EC1F
:1049FF00FEE493FFEEC39F5026AE5AAF5B0FBF008E
:104A0F00010E907116120048AE5AAF5BE493FC9002
:104A1F007116120048E493900091127310ECF0AEEF
:104A2F005AAF5B907116120048E493900091127385
:104A3F0010E0FC907118120048ECFCE493FDECD3ED
:104A4F009D4019907118120048E493FC9071161252
:104A5F000048E493900091127310ECF0AE5AAF5BE4
:104A6F00742D6F4E7006755B33755A00AE5AAF5B7F
:104A7F0074022FFF50010E8E5A8F5B785B740126E4
:104A8F00F6500418E436F640030249D42285F9742F
:104A9F0085FA757E017F00E5751272DFE5742FFFD1
:104AAF0050010E8E5A8F5BAC5CAD5DEF2DFDEE3C71
:104ABF00FC8C5C8D5D123D78123D83123D8E123D54
:104ACF00999000D9E0D39402402C75A71085F97402
:104ADF0085FA757E017F00E5751272DFE5742FFF91
:104AEF0050010E8E5A8F5B123DA4123DBB123DD268
:104AFF00123DED75A7002275A71085F97485FA751B
:104B0F007E017F00E5751272DFE5742FFF50010EF5
:104B1F008E5A8F5B7E017F76900116E01272DFACAA
:104B2F005AAD5BED2FFFEC3EFE8E5C8F5DE55DF5C4
:104B3F00FDE55CF5FE900082E4F075A7007412901D
:104B4F00005FF02285F97485FA757E017F00E575A7
:104B5F001272DFE5742FFF50010E8E5A8F5B90009B
:104B6F0018E0FCA3E0FDEF2DFDEE3CFC8C5C8D5DB1
:104B7F00E55DF5FDE55CF5FE22056522A2D8B340A3
:104B8F0002C293A2D9B34002C294A2DAB34002C2C6
:104B9F0091A2DBB34002C292A2DCB34030A2965086
:104BAF0006741990005FF0A2955006741990005F7B
:104BBF00F0A2A05006741990005FF0A297500674EF
:104BCF001990005FF0C296C295C2A0C29775D840E7
:104BDF002285A77375A710A2D8B34002C287A2D9A6
:104BEF00B34002C290A2DAB34006E5B554EFF5B573
:104BFF00A2DBB34006E5B554DFF5B5A2DCB3400840
:104C0F009000E5E0900082F075D8408573A7229060
:104C1F00F800E4936406600280FE12009E75A70000
:104C2F0075D80075D90475DA0975DB0975DC097556
:104C3F00DD0975DE0975D84075A71075D80075D9CF
:104C4F000475DA0975DB0975DC0975DD0975DE098F
:104C5F0075D84075A7001200FB74C8F509750800D8
:104C6F001205E475A70FE5FC90006EF0E5FB9000D0
:104C7F006FF0E5FA900070F0E5F9900071F075A70C
:104C8F000090F800E493F5281207039008A8E0D3EA
:104C9F00940350079008A8E0B4010674009008A888
:104CAF00F09008A8E09008FFF074019000DAF090FF
:104CBF0008A8E0906BCAF8282873802A802875A767
:104CCF000F75F30F75A700A2A3400674029000DAC8
:104CDF00F0801375A70F75F31775A700A2A44006F0
:064CEF0074029000DAF0EF
:0C6BCA00024CC9024CCB024CCD024CE244
:104CF5009000DAE0B4022AC21A120AAC74029000DB
:104D0500DAF09008A8E0906BD6F828287380108018
:0F4D15000E74009000E9F0800674009000F6F034
:0C6BD600024D12024D14024D16024D1E1D
:104D24008028D21A1209C174019000DAF09008A800
:104D3400E0906BE2F82828738010800E74009000D5
:0A4D4400E9F0800674009000F6F01C
:0C6BE200024D3C024D3E024D40024D4869
:104D4E0090F807E49390007BF090007BE04408908D
:104D5E00007BF090007BE054FE90007BF012039DF0
:104D6E00123EC09008B5E090017DF09008B6E0903C
:104D7E00017EF09008B7E090017FF090017DE07029
:104D8E000C90017EE0700690017FE060028004C20C
:104D9E00258002D2259000CBE004900086F01248C8
:104DAE000B90F802E493B405051249CE8003124924
:104DBE00007400900101F0124007E5B54401F5B50D
:104DCE007406900061F07400900062F0740190001F
:104DDE0063F090F802E493900064F090F803E4938B
:104DEE00900065F090F804E493900066F0740690DD
:104DFE000067F0900064E0B405067405900067F05B
:104E0E00742B900068F07403900069F074069000A3
:104E1E006AF0740790006BF090F805E49390006CC4
:104E2E00F090F806E49390006DF07400900075F029
:104E3E007400900076F07400900077F0740090008B
:104E4E0078F07400900079F0740090007AF074FF9E
:104E5E0090007CF0A2B6B39205A2B3B39206A2A4C0
:104E6E00B39222A2A3B3922390007DE4F07570005A
:104E7E00743A900791F074FD900792F090007EE4E2
:104E8E00F0756F0190005FE4F09000DBE0B4010676
:104E9E00741A90005FF0C221756400C20AD20BC270
:104EAE0003757200C224120586756000756C00755C
:104EBE006200756632756700756800756900756AFF
:104ECE0000756B0090001EE4F0A3F0756D00D2B279
:104EDE00D2A4D2B0D2B1D2A3D2A7D2A6D2A5D2B7E3
:104EEE007E017F009000B8E01272DF9000B7E02FD5
:104EFE00FF50010E900028EEF0A3EFF0EFD394FFD9
:104F0E00EE940F4007900028E4F0A3F0900100E02B
:104F1E00700674FF900100F09000DBE07005756E76
:104F2E00028003756E03741990011EF0741A9001BD
:104F3E001FF0742A900120F07400900121F074008B
:104F4E009006F3F074009006F4F074009006F7F0FB
:104F5E0074009006F8F074009006FBF07400900652
:104F6E00FCF0741590077FF07416900780F074179C
:104F7E00900781F07418900782F07400900783F008
:104F8E007400900784F07400900785F07400900709
:104F9E0086F07401900787F07402900788F074030E
:104FAE00900789F0740490078AF0D29CE571D3942F
:104FBE001040037571109006D8E0D3940C4006741F
:104FCE00009006D8F09006DCE0D3940C40067400F6
:104FDE009006DCF09006E0E0D3940C40067400904E
:104FEE0006E0F09006E4E0D3940C400674009006C0
:104FFE00E4F09006E8E0D3940C400674009006E8C6
:10500E00F09006ECE0D3940C400674009006ECF0A1
:10501E009006F0E0D3940C400674009006F0F0D2A7
:10502E00EC75CF01A298B34005C298120C14E54E50
:10503E006006A299B3B340028005C2991210A3E58F
:10504E004F64016005E54FB4040280D5C28E7E1018
:10505E007F00E5651272DFE58D75F010A4FDACF0F2
:10506E00EF2DFDEE3CFCE58B75F01084FF7E00ED20
:10507E002FFFEC3EFE8E548F55D28E9000BEE06018
:10508E00099000BEE0C3943D4002805C9000201267
:10509E0072ED900020E0FEA3E0FF900022E0FCA362
:1050AE00E0FDEFB50542EEB5043EB218A204B340E2
:1050BE001975E700A218B34008E5B54404F5B580AC
:1050CE0006E5B554FBF5B575E710900022E0FEA39A
:1050DE00E0FF900024E0FCA3E0FDEF2DFDEE3CFC94
:1050EE00900022ECF0A3EDF09000CBE06009900070
:1050FE00CBE0C394034002807D122FCEA204400861
:10510E009000B5E0F546801BE560C39561500575CE
:10511E004600800F9000A2E0C3956250069000C832
:10512E00E0F546E54675F002A4FFAEF090089DEE60
:10513E00F0A3EFF075E700AC2FAD30EDD39FEC9EF2
:10514E004015E5B5547FF5B59000CBE0B40206E509
:10515E00B54440F5B5801C90007DE0C394415013DA
:10516E00E5B54480F5B59000CBE0B40206E5B55444
:10517E00BFF5B575E7109000CBE0B4032A1230E905
:10518E0075E700AE2FAF3090089DE0FCA3E0FDEF79
:10519E00D39DEE9C4008E5B54480F5B58006E5B597
:1051AE00547FF5B575E7109000A6E06009A2B33004
:1051BE000601B3B340028028A2B3300601B34020EB
:1051CE00A2B3300801B3400B90008DE004F0A208AA
:1051DE00B39206A208B330B301B34004A2089206FC
:1051EE00A2B6300501B3500302587CA2B6300501B9
:1051FE00B3500302587CA2B6300701B350030257D6
:10520E004C756F009000BEE0B43D1975E700A20723
:10521E00B34008E5B554FBF5B58006E5B54404F595
:10522E00B575E710055FA209B3B35013AE54AF5571
:10523E00900010E0FCA3E0FDEDC39FEC9E40030246
:10524E0053F9E56EB40375A229B34022E55FB4129B
:10525E0003756E01E55FC39412500690005F7401F2
:10526E00F0E55FD394124006740290005FF0900058
:10527E008DE06401600790008DE0B40405755F0158
:10528E00801A90008DE06402600790008DE0B403F8
:10529E0005755F138006740590005FF090008DE039
:1052AE00B40102D21E90008DE0B40402C21ED229B7
:1052BE0090008DE0B40102D21E02536BE56EB40273
:1052CE0006756E01755F12E55F64126005E55FB4E9
:1052DE00244290008DE06401600790008DE0B404DC
:1052EE0005755F01801A90008DE0640260079000E2
:1052FE008DE0B40305755F138006740590005FF0B2
:10530E0090008DE0B40102D21E90008DE0B4040234
:10531E00C21E804990005FE07034E55FC394125066
:10532E000690005F7401F0E55FD39412400674029C
:10533E0090005FF0E55FC394125002D221E55FD377
:10534E0094124002D221C296C295C2A0C29790007A
:10535E00DBE0B401051247198003755F01AE56AF4D
:10536E0057AC54AD55EF2DFDEE3CFC7403FF12729D
:10537E00CF8C568D579000BEE060099000BEE0C302
:10538E00943D40028049900020E0FEA3E0FF900093
:10539E00BEE08E048F05FF1272CF74018C068D074E
:1053AE00120039900024EEF0A3EFF0900024E0F804
:1053BE00A3E0900022C8F0A3C8F0900020E4F0A370
:1053CE00F0C21875E700E5B554FBF5B575E710A208
:1053DE00A4B34002C222A2A3B34002C223A221B3AD
:1053EE004002C22190008DE4F0803AAE56AF57AC29
:1053FE0054AD55EF2DFDEE3CFC74018C068D07125D
:10540E0000398E568F57E56EC39402500DAC54ADD5
:10541E00557488C39D74139C4002800912471974F9
:10542E000690005FF0E55FB41212740390005FF017
:10543E00D2219000DBE0B40103124719AE58AF59E8
:10544E00AC54AD55EF2DFDEE3CFC8C588D59AE5441
:10545E00AF55EFD39DEE9C4011900016E0FAA3E0FD
:10546E00FBEBC394E8EA9403400280069000161208
:10547E0072ED900014E0FEA3E0FFAC54AD55EF2D9D
:10548E00FDEE3CFC900014ECF0A3EDF09000DBE0A0
:10549E00B4011DAE54AF5574051272DF74038E0441
:1054AE008F05FF1272CF900010ECF0A3EDF0801676
:1054BE00AE54AF5574031272DF74011200399000AE
:1054CE0010EEF0A3EFF0C28E758D00758B00756532
:1054DE0000755501755400D28EE55F240875F009EC
:1054EE0084AFF07E00EF4E600302557CE56E6013D4
:1054FE00AE56AF5774091272DF900012EEF0A3EFA2
:10550E00F0800F900014E0F8A3E0900012C8F0A312
:10551E00C8F0900012E0FEA3E0FFEF4E600B7C7F20
:10552E007D7E1271CD8E528F53900014E4F0A3F055
:10553E00AE52AF537428BE00039F5010E5642FFF88
:10554E0050010E74011200398E528F5385536490A0
:10555E0000E2E0A852B8000DD395534008E55390F1
:10556E00005EF080099000E2E01490005EF0900082
:10557E00D9E0B40308900052E0655F6002800EA28D
:10558E001E301F01B34004D2208002C220E55F64AA
:10559E000B6005E55FB41D099000CBE06003122C93
:1055AE008490005CE0655F600790005DE0B55F038E
:1055BE00757000A20AB35006A209B3B34003025697
:1055CE0074900097E0B40173900119E0B4021412C4
:1055DE001244900083E075F0BCA4FFAEF08E5C8F99
:1055EE005D8056E56875F00A84FF7E009005911285
:1055FE000048E0F55B755A00AE5AAF5B9000BCE018
:10560E001272DF74648E048F05FF1272CF8C5C8D64
:10561E005DE55D90005AF0AE5AAF5B900095E012DA
:10562E0072DF74648E048F05FF1272CF74BC8C0609
:10563E008D071272DF8E5C8F5D8017900095E0757E
:10564E00F0BCA4FFAEF08E5C8F5D9000BCE09000CD
:10565E005AF0E562C394CC5006E55D455C7002805D
:10566E0003124A9CD20AE56EB40106E55F640B6034
:10567E0002800C7571009000607401F0756E00E58B
:10568E006E60030257479000DEE0600D900082E0EE
:10569E00A852B800069553400280489000DEE0B450
:1056AE00022790004EE0655F601790004FE0655F47
:1056BE00600F900050E0655F6007900051E0B55FAD
:1056CE0003757103756D00800CC201756D0090003D
:1056DE001EE4F0A3F0900082E06006740990005F73
:1056EE00F0805690004EE0655F601790004FE065C9
:1056FE005F600F900050E0655F6007900051E0B56D
:10570E005F3775710090004EE0B55F0690006074D3
:10571E0001F090004FE0B55F067402900060F090CB
:10572E000050E0B55F067403900060F0900051E009
:10573E00B55F067404900060F0A207B39205A2074D
:10574E00B330B601B3500302587C756F019000BEA2
:10575E00E0B43D1975E700A207B34008E5B544046F
:10576E00F5B58006E5B554FBF5B575E71075E700A0
:10577E00E5B54401F5B575E710742B90007DF0A2E8
:10578E00079205E55FD3944A4014D209E55FD3949E
:10579E006E400B740590005FF0D221755F4675E781
:1057AE0000900114E0A852B80005D39553500D9007
:1057BE000113E0A852B80004955350028008E5B5D5
:1057CE004402F5B58017900115E0D395624008E5C7
:1057DE00B54402F5B58006E5B554FDF5B575E7108F
:1057EE009000E6E0B40107E56BC3944140028018D7
:1057FE00E56BC394145008741390005FF080067428
:10580E000E90005FF0124719900067E0FE90006462
:10581E00E0C39E4009900064E0D39408400974FBF5
:10582E0090005FF0124719900065E06015900065DA
:10583E00E0FE900063E06E600974FC90005FF01271
:10584E004719900066E06015900066E0FE900068D3
:10585E00E06E600974FE90005FF01247199008A880
:10586E00E06006900116E060028003120B97A22101
:10587E00B34008C296C295C2A0C297900116E060CE
:10588E000CAE52AF537414BE00059F400280379089
:10589E00009EE0906BEEF8282873802A8028A2A341
:1058AE00B35005A223B340028005124B06D22380CB
:1058BE0015A2A4B35005A222B340028005124B06D6
:0658CE00D22280028000DE
:106BEE000258A80258AA0258AC0258BF0258D20244
:026BFE0058D469
:1058D400A20CB3B35008900052E0655F6003025A13
:1058E4005AA202B35006A201B3B34003025A529023
:1058F40000D9E0B404028003025A0F9008FBE0B41C
:10590400020280030259F4A220B3406A123CD890E8
:10591400012AE0601F90001CE0FEA3E0FF9001223A
:10592400E01272DF74C88E048F05FF1272CF8C5C94
:105934008D5D800A90001CE0F55CA3E0F55DAE5C33
:10594400AF5D745E1272DF74058E048F05FF1272F0
:10595400CFAE5AAF5BED2FFFEC3EFE8E5C8F5D90B9
:10596400003CE0FCA3E0FDEF2DFDEE3CFC8C5C8DE7
:105974005D123D78806E123D1790012AE0D39404A5
:10598400401F90001CE0FEA3E0FF900126E012728D
:10599400DF74C88E048F05FF1272CF8C5C8D5D801E
:1059A4000A90001CE0F55CA3E0F55DAE5CAF5D74AD
:1059B4005E1272DF74058E048F05FF1272CFAE5A29
:1059C400AF5BED2FFFEC3EFE8E5C8F5D90003CE004
:1059D400FCA3E0FDEF2DFDEE3CFC8C5C8D5D123DE7
:1059E400A475A7009000F7E0B40103123E088019E3
:1059F400123CD8123D78123D17123DA475A70090B1
:105A040000F7E0B40103123E088043123CD8123D73
:105A1400789000D9E0B4031275A710123DA4900049
:105A2400F7E0B40103123E08802175A7109000F737
:105A3400E0B40106A203B3B340028005123DA48082
:105A44000A9000F7E0B40203123DA475A700C20C4B
:105A5400D20DD20ED20FA20DB3B35008900053E072
:105A6400655F6003025BE3A202B35006A201B3B315
:105A74004003025BDB9000D9E0B404028003025BC4
:105A8400989008FBE0B402028003025B7DA220B37D
:105A9400406D123CD890012AE0D39401401F90003D
:105AA4001CE0FEA3E0FF900123E01272DF74C88EB5
:105AB400048F05FF1272CF8C5C8D5D800A90001CF0
:105AC400E0F55CA3E0F55DAE5CAF5D745E1272DF81
:105AD40074058E048F05FF1272CFAE5AAF5BED2FA3
:105AE400FFEC3EFE8E5C8F5D90003CE0FCA3E0FD8D
:105AF400EF2DFDEE3CFC8C5C8D5D123D83806E12BF
:105B04003D1790012AE0D39405401F90001CE0FE4D
:105B1400A3E0FF900127E01272DF74C88E048F05A2
:105B2400FF1272CF8C5C8D5D800A90001CE0F55CE6
:105B3400A3E0F55DAE5CAF5D745E1272DF74058E3A
:105B4400048F05FF1272CFAE5AAF5BED2FFFEC3E10
:105B5400FE8E5C8F5D90003CE0FCA3E0FDEF2DFD2C
:105B6400EE3CFC8C5C8D5D123DBB75A7009000F78C
:105B7400E0B40103123E088019123CD8123D83128E
:105B84003D17123DBB75A7009000F7E0B401031266
:105B94003E088043123CD8123D839000D9E0B40300
:105BA4001275A710123DBB9000F7E0B40103123E3A
:105BB40008802175A7109000F7E0B40106A203B392
:105BC400B340028005123DBB800A9000F7E0B402A6
:105BD40003123DBB75A700D20CC20DD20ED20FA288
:105BE4000EB3B35008900054E0655F6003025D6C2F
:105BF400A202B35006A201B3B34003025D64900055
:105C0400D9E0B404028003025D219008FBE0B402F1
:105C1400028003025D06A220B3406D123CD89001BD
:105C24002AE0D39403401F90001CE0FEA3E0FF9001
:105C34000124E01272DF74C88E048F05FF1272CF44
:105C44008C5C8D5D800A90001CE0F55CA3E0F55D42
:105C5400AE5CAF5D745E1272DF74058E048F05FF57
:105C64001272CFAE5AAF5BED2FFFEC3EFE8E5C8F0F
:105C74005D90003CE0FCA3E0FDEF2DFDEE3CFC8CD0
:105C84005C8D5D123D8E806E123D1790012AE0D32B
:105C94009406401F90001CE0FEA3E0FF900128E062
:105CA4001272DF74C88E048F05FF1272CF8C5C8D64
:105CB4005D800A90001CE0F55CA3E0F55DAE5CAF8E
:105CC4005D745E1272DF74058E048F05FF1272CF4D
:105CD400AE5AAF5BED2FFFEC3EFE8E5C8F5D900005
:105CE4003CE0FCA3E0FDEF2DFDEE3CFC8C5C8D5D07
:105CF400123DD275A7009000F7E0B40103123E08EC
:105D04008019123CD8123D8E123D17123DD275A750
:105D1400009000F7E0B40103123E088043123CD81F
:105D2400123D8E9000D9E0B4031275A710123DD233
:105D34009000F7E0B40103123E08802175A710908B
:105D440000F7E0B40106A203B3B340028005123D9C
:105D5400D2800A9000F7E0B40203123DD275A70086
:105D6400D20CD20DC20ED20FA20FB3B350089000C2
:105D740055E0655F6003025EF5A202B35006A2011E
:105D8400B3B34003025EED9000D9E0B40402800393
:105D9400025EAA9008FBE0B402028003025E8FA2B6
:105DA40020B3406D123CD890012AE0D39403401FE5
:105DB40090001CE0FEA3E0FF900125E01272DF7466
:105DC400C88E048F05FF1272CF8C5C8D5D800A90A3
:105DD400001CE0F55CA3E0F55DAE5CAF5D745E12A3
:105DE40072DF74058E048F05FF1272CFAE5AAF5B5B
:105DF400ED2FFFEC3EFE8E5C8F5D90003CE0FCA33B
:105E0400E0FDEF2DFDEE3CFC8C5C8D5D123D998038
:105E14006E123D1790012AE0D39407401F90001C96
:105E2400E0FEA3E0FF900129E01272DF74C88E0443
:105E34008F05FF1272CF8C5C8D5D800A90001CE090
:105E4400F55CA3E0F55DAE5CAF5D745E1272DF7469
:105E5400058E048F05FF1272CFAE5AAF5BED2FFF94
:105E6400EC3EFE8E5C8F5D90003CE0FCA3E0FDEF19
:105E74002DFDEE3CFC8C5C8D5D123DED75A7009014
:105E840000F7E0B40103123E088019123CD8123D19
:105E940099123D17123DED75A7009000F7E0B4018B
:105EA40003123E088043123CD8123D999000D9E079
:105EB400B4031275A710123DED9000F7E0B401038E
:105EC400123E08802175A7109000F7E0B40106A2E5
:105ED40003B3B340028005123DED800A9000F7E061
:105EE400B40203123DED75A700D20CD20DD20EC23E
:0E5EF4000FE571906C00F82828739000FEE016
:036C0000025EFE33
:105F0200906C33F82828731225CF80121225CF8087
:0E5F12000D122659800812270580031227055C
:0F6C3300025F09025F0E025F13025F18025F1D0E
:105F20007571010264031228311229487571020249
:105F30006403122CC8A204B340139000E3E075F090
:105F40001DA4FFAEF0900018EEF0A3EFF0900891C2
:105F5000E0FEA3E0FF740A1272DF900012E0FCA3DF
:105F6000E0FD74098F02FF1272CF8D078C038E043F
:105F70008A058B061271CD900895EEF0A3EFF074B0
:105F8000F0BE00039F500B74F0900895F8E4F0E821
:105F9000A3F0E5377003753701900895E0FEA3E0A4
:105FA000FFE5372FFF50010E900895EEF0A3EFF0BC
:0B5FB000757103A230401F900060E0FC
:066C0300025F26025F3271
:105FBB00906C42F8282873801275710A800D7571E8
:0B5FCB000B800875710C800375710DD0
:0F6C4200025FC2025FC4025FC9025FCE025FD36E
:105FD6000264039006D8E06006750801122DF6A249
:105FE60032B3401675E70090078FE0B42906E5B591
:105FF6004408F5B575E7100260A19000CCE0D39493
:106006000240459000A0E02403A852B8000495532E
:1060160050099000A2E0D395625002800ED202A2EF
:10602600284006740890005FF0D2289000A0E0A8EF
:1060360052B80005D39553500B9000A2E02403C339
:1060460095625002C20280539000A0E02403A85239
:10605600B8000495535010E560C39561500990004F
:10606600A2E0D395625002800ED202A228400674A6
:106076000890005FF0D2289000A0E0A852B8000572
:10608600D395535014E561240FC39560400B9000DF
:10609600A2E02403C395625002C202A2024002C2D9
:1060A60028A232B35005A202B34002801375E7005E
:1060B60090078FE0B42906E5B554F7F5B575E710F6
:1060C6009000E6E07007E56BC3941440028002D2AC
:1060D600029000DBE0B40102D202A2024005757113
:1060E60004800A75711090001EE4F0A3F0026403A8
:0460F6009000CCE06A
:066C0900025FD90260F6F3
:1060FA00906C51F828287312135A801212135A807E
:0E610A000D12150D80081215C480031215C465
:0F6C510002610102610602610B0261100261150E
:106118009006DCE06006750802122DF6757105021E
:10612800640312171D7571069006E0E06006750895
:1061380003122DF69006E4E06006750804122DF6A9
:1061480002640390005AE06006A204B3B3400280E0
:106158000DE55FD39409500690005AE014F0121927
:10616800A67571079006E8E06006750805122DF619
:106178009006ECE06006750806122DF6026403909E
:106188000119E0B402031212CB121E0E75710890A9
:1061980006F0E06006750807122DF6026403121E69
:1061A800F07571090264031222C8A20CB35005A24B
:1061B8000DB340028008D20CD20DD20ED20F7571E9
:1061C80010026403900040E0C394465008C29674DD
:1061D80046900040F0900056E0B4011DE537240ACF
:1061E800F537900895E0FEA3E0FF740A2FFF5001F1
:1061F8000E900895EEF0A3EFF085375B755A009086
:10620800004EE0F574123F80E55D900040F090008C
:1062180008E55AF0A3E55BF0E574900041F0C2117F
:10622800900895E0F55AA3E0F55B90004EE0F57410
:10623800123F80E55D90003EF0900000E55AF0A323
:10624800E55BF0E57490003FF0C2107571030264DD
:1062580003900044E0C394465008C29574469000E9
:1062680044F0900057E0B4011DE537240AF5379053
:106278000895E0FEA3E0FF740A2FFF50010E900876
:1062880095EEF0A3EFF085375B755A0090004FE06C
:10629800F574123F80E55D900044F090000AE55ADD
:1062A800F0A3E55BF0E574900045F0C21390089503
:1062B800E0F55AA3E0F55B90004FE0F574123F80DB
:1062C800E55D900042F0900002E55AF0A3E55BF02E
:1062D800E574900043F0C2127571030264039000E4
:1062E80048E0C394465008C2A07446900048F09015
:1062F8000058E0B4011DE537240AF537900895E009
:10630800FEA3E0FF740A2FFF50010E900895EEF0EF
:10631800A3EFF085375B755A00900050E0F57412D2
:106328003F80E55D900048F090000CE55AF0A3E549
:106338005BF0E574900049F0C215900895E0F55AB5
:10634800A3E0F55B900050E0F574123F80E55D90A6
:106358000046F0900004E55AF0A3E55BF0E5749080
:106368000047F0C21475710302640390004CE0C347
:1063780094465008C297744690004CF0900059E03B
:10638800B4011DE537240AF537900895E0FEA3E02F
:10639800FF740A2FFF50010E900895EEF0A3EFF05E
:1063A80085375B755A00900051E0F574123F80E51F
:1063B8005D90004CF090000EE55AF0A3E55BF0E527
:1063C8007490004DF0C217900895E0F55AA3E0F5D7
:1063D8005B900051E0F574123F80E55D90004AF053
:1063E800900006E55AF0A3E55BF0E57490004BF0E9
:0B63F800C21675710380048002800053
:106C0F0002612A02614B0261870261A60261AF0233
:106C1F0061CC0262590262E60263730263FF02648F
:046C2F0001026403F7
:1064030090003EE0B55F73A210404F900000E0FEA5
:10641300A3E0FFEF4E6021AE56AF57900000E0FCC3
:10642300A3E0FD120003740A8E048F05FF1272CFDE
:10643300900000ECF0A3EDF090003FE0601A9000B4
:1064430000E0FEA3E0FFAC56AD57EF2DFDEE3CFCA4
:10645300900000ECF0A3EDF0D210AE54AF559000D5
:1064630000E0FCA3E0FDEFC39DEE9C400D124B53F7
:10647300D296C21074C890003EF0A210B3B3500776
:1064830090003EE0B55F02800D124B53D29674C864
:1064930090003EF0C210900040E0B55F70A2114042
:1064A3004F900008E0FEA3E0FFEF4E6021AE56AF31
:1064B30057900008E0FCA3E0FD120003740A8E0469
:1064C3008F05FF1272CF900008ECF0A3EDF090005F
:1064D30041E0601A900008E0FEA3E0FFAC56AD5720
:1064E300EF2DFDEE3CFC900008ECF0A3EDF0D21193
:1064F300AE54AF55900008E0FCA3E0FDEFC39DEE62
:106503009C400AC2967446900040F0C211A211B397
:10651300B35007900040E0B55F02800AC29674460C
:10652300900040F0C211900042E0B55F73A21240A8
:106533004F900002E0FEA3E0FFEF4E6021AE56AFA6
:1065430057900002E0FCA3E0FD120003740A8E04DE
:106553008F05FF1272CF900002ECF0A3EDF09000D4
:1065630043E0601A900002E0FEA3E0FFAC56AD5793
:10657300EF2DFDEE3CFC900002ECF0A3EDF0D21207
:10658300AE54AF55900002E0FCA3E0FDEFC39DEED7
:106593009C400D124B53D295C21274C8900042F026
:1065A300A212B3B35007900042E0B55F02800D1210
:1065B3004B53D29574C8900042F0C212900044E04D
:1065C300B55F70A213404F90000AE0FEA3E0FFEF17
:1065D3004E6021AE56AF5790000AE0FCA3E0FD12D7
:1065E3000003740A8E048F05FF1272CF90000AEC29
:1065F300F0A3EDF0900045E0601A90000AE0FEA3DE
:10660300E0FFAC56AD57EF2DFDEE3CFC90000AECDD
:10661300F0A3EDF0D213AE54AF5590000AE0FCA303
:10662300E0FDEFC39DEE9C400AC295744690004482
:10663300F0C213A213B3B35007900044E0B55F0256
:10664300800AC2957446900044F0C213900046E05D
:10665300B55F73A214404F900004E0FEA3E0FFEF88
:106663004E6021AE56AF57900004E0FCA3E0FD124C
:106673000003740A8E048F05FF1272CF900004EC9E
:10668300F0A3EDF0900047E0601A900004E0FEA351
:10669300E0FFAC56AD57EF2DFDEE3CFC900004EC53
:1066A300F0A3EDF0D214AE54AF55900004E0FCA378
:1066B300E0FDEFC39DEE9C400D124B53D2A0C214DC
:1066C30074C8900046F0A214B3B35007900046E09C
:1066D300B55F02800D124B53D2A074C8900046F0F0
:1066E300C214900048E0B55F70A215404F90000CB3
:1066F300E0FEA3E0FFEF4E6021AE56AF5790000CD3
:10670300E0FCA3E0FD120003740A8E048F05FF1260
:1067130072CF90000CECF0A3EDF0900049E0601A0A
:1067230090000CE0FEA3E0FFAC56AD57EF2DFDEE5D
:106733003CFC90000CECF0A3EDF0D215AE54AF5539
:1067430090000CE0FCA3E0FDEFC39DEE9C400AC269
:10675300A07446900048F0C215A215B3B350079039
:106763000048E0B55F02800AC2A07446900048F07A
:10677300C21590004AE0B55F73A216404F90000621
:10678300E0FEA3E0FFEF4E6021AE56AF5790000648
:10679300E0FCA3E0FD120003740A8E048F05FF12D0
:1067A30072CF900006ECF0A3EDF090004BE0601A7E
:1067B300900006E0FEA3E0FFAC56AD57EF2DFDEED3
:1067C3003CFC900006ECF0A3EDF0D216AE54AF55AE
:1067D300900006E0FCA3E0FDEFC39DEE9C400D128C
:1067E3004B53D297C21674C890004AF0A216B3B3A3
:1067F300500790004AE0B55F02800D124B53D297C9
:1068030074C890004AF0C21690004CE0B55F70A2C5
:1068130017404F90000EE0FEA3E0FFEF4E6021AE65
:1068230056AF5790000EE0FCA3E0FD120003740A7C
:106833008E048F05FF1272CF90000EECF0A3EDF0E3
:1068430090004DE0601A90000EE0FEA3E0FFAC560E
:10685300AD57EF2DFDEE3CFC90000EECF0A3EDF0F8
:10686300D217AE54AF5590000EE0FCA3E0FDEFC38A
:106873009DEE9C400AC297744690004CF0C217A24A
:1068830017B3B3500790004CE0B55F02800AC2977C
:10689300744690004CF0C2179000E9E0B402028005
:1068A300030269CF90007FE0D39567506490007F27
:1068B300E0F4042567FE9000ECE08E00F5F0E88438
:1068C300FF7E008F74EFC39410500CEF8574F0A417
:1068D300FDACF08D7480037574FF90007FE0D39559
:1068E30074400B90007FE0C39574F572800375725A
:1068F30000900107E0D395724006900107E0F5721E
:10690300900108E0C395725006900108E0F572808B
:106913007190007FE0C39567FE9000ECE08E00F578
:10692300F0E884FF7E008F74EFC39410500CEF8562
:1069330074F0A4FDACF08D7480037574FF85745BF3
:10694300755A0090007FE0255BFFAE5A50010E8E12
:106953005A8F5B74FFBE0009D39F4005855B72802D
:10696300037572FF900107E0D3957240069001070B
:10697300E0F572900108E0C395725006900108E0BB
:10698300F572A204B3B3500D900080E0FE9000F4C2
:10699300E0D39E50028014740790005FF075E70007
:1069A300E5B554BFF5B575E710802175A71075E7F8
:1069B30000E5CDC395724008E5B554BFF5B5800633
:1069C300E5B54440F5B575E71075A70090010EE0F5
:1069D300A852B800049553501790010DE0A852B87F
:1069E300000ED39553400990010FE0D39562400206
:1069F300801975A710E5CDC394BF4004C2A28002DD
:106A0300D2A2A2A292A175A700801775A710E5CD07
:106A1300C394404004C2A28002D2A2A2A292A17552
:106A2300A700E570C39413501DE57075F00284AFA1
:106A3300F07E00EF4E7005123290800AA2EDB34053
:106A430005C2ED123290AE54AF557410C39F742734
:106A53009E400C90007EE0C3945A4003026BAFA2A9
:106A630009B34009124719740690005FF0A20BB3F3
:106A7300500EE562D394334007E562C394CC4002E1
:106A83008041900119E0B40214121244900083E093
:106A930075F05EA4FFAEF08E5C8F5D800F90009565
:106AA300E075F05EA4FFAEF08E5C8F5DE55D455C46
:106AB3006011E5B54401F5B5742B90007DF0124AE1
:106AC3009CD20B90007EE0D394014007E562C3940F
:106AD3001A40028002C20B9006D8E06006750801D6
:106AE300122DF69006DCE06006750802122DF69072
:106AF30006E0E06006750803122DF69006E4E060F8
:106B030006750804122DF69006E8E0600675080580
:106B1300122DF69006ECE06006750806122DF6902D
:106B230006F0E06006750807122DF690007EE0C3BC
:106B3300945A5010E570B4130990007EE004F07588
:106B43007000803FE570B41303757000C28E758DBD
:106B530000758B00756500755501755400D28E90D4
:106B6300007DE0C39441500890007DE004F080066E
:106B7300744190007DF090007DE0B44106E5B5548A
:106B8300FEF5B590007EE0D394014007E56BC39416
:106B93004140028006740E90005FF09008A8E06008
:0F6BA30006900116E060028003120B9702502F3C
:106C60000000010001400160018001A001C001E0BD
:106C700002000300039603B603D603F404000500E4
:106C80000512052405360548055A056C057E059054
:106C900005A805C005DE0600061406280646066E91
:106CA00006AE05CF06EE00FF013F015F017F019FA9
:106CB00001BF01DF01FF02FF039503B503D503F315
:106CC00003FF04FF05110523053505470559056B2D
:106CD000057D058F05A705BF05CE05F1061306271F
:106CE0000645066D06AD06ED05DD06FF0FAA0FA5EC
:106CF0000F9F0F9A0F940F8D0F870F800F780F71D2
:106D00000F680F600F570F4E0F450F3B0F300F25C9
:106D10000F1A0F0E0F020EF50EE80EDB0ECC0EBE94
:106D20000EAE0E9F0E8E0E7D0E6C0E5A0E470E345A
:106D30000E200E0C0DF70DE20DCB0DB50D9D0D8542
:106D40000D6D0D540D3A0D200D050CE90CCE0CB156
:106D50000C940C760C580C3A0C1B0BFB0BDB0BBB8E
:106D60000B9A0B790B570B350B130AF10ACE0AABB2
:106D70000A870A640A400A1C09F809D409B0098C78
:106D800009670943091F08FB08D608B2088E086A7C
:106D90000846082307FF07DC07B907960773075162
:106DA000072F070D06EC06CA06AA068906690649DA
:106DB000062A060A05EC05CD05B0059205750558AD
:106DC000053C0520050504EA04CF04B5049C0482B3
:106DD0000469045104390422040B03F403DE03C8DC
:106DE00003B2039D038903750361034D033B03282D
:106DF0000316030402F202E102D102C002B002A0B3
:106E0000029102820273026502570249023C022F7C
:106E100002220216020901FD01F201E601DB01D0A6
:106E200001C601BB01B101A7019D0194018B018243
:106E30000179017001680160015801500148014168
:106E400001390132012B0125011E01180111010B2D
:106E5000010500FF00FA0FA60FA00F990F920F8BEC
:106E60000F840F7C0F740F6B0F620F580F4E0F4380
:106E70000F380F2C0F1F0F120F050EF70EE80ED84C
:106E80000EC80EB70EA50E930E800E6C0E580E4255
:106E90000E2C0E150DFD0DE40DCB0DB10D950D79DC
:106EA0000D5D0D3F0D200D010CE10CC00C9E0C7C06
:106EB0000C590C350C100BEA0BC40B9E0B760B4FC8
:106EC0000B260AFD0AD40AAA0A800A550A2A09FFD3
:106ED00009D409A8097C0950092508F908CD08A199
:106EE0000875084A081E07F307C8079D0773074976
:106EF000072006F706CE06A6067E06570630060AC7
:106F000005E405BF059B057705540532051004EF20
:106F100004CE04AE048F047104530435041903FD38
:106F200003E203C703AD0394037B0363034B033402
:106F3000031E030802F302DE02CA02B602A3029194
:106F4000027F026D025C024C023C022C021D020E0A
:106F5000020001F201E401D701CA01BE01B101A69C
:106F6000019A018F0185017A01700166015D01536B
:106F7000014A01410139013101290121011901129F
:106F8000010B010400FD00F700F000EA00E400DE60
:106F900000D900D300CE00C900C400BF00BA00B5BC
:106FA00000B100AD00A800A400A0009C00990095CD
:106FB0000091008E008A008700840081007E007BA3
:10009E0075B50075840175A70075FFA075EF069004
:1000AE00005BE4F075C91075A70F75A1C775A700A1
:1000BE0075D90075CE0C75A70F75F1FE75F2FF752B
:1000CE00F30775F47875A4BA75A5FF75A60775AE16
:1000DE000075AFFF75D48175D5FF75D6FF75D7FF47
:1000EE0075A70075A20175A14775F8092275E60876
:1000FE0075E71075BC0175BE0475BD6C75BE0775D0
:10010E00BDA075BE0875BD0175BC0075BB1875BC6C
:10011E002075BA0875E88075D11375A70F75E105BE
:10012E0075E20075C7401247197597007597807470
:10013E000A1272BF7597C0E5975420700280F87549
:10014E008F0275A700D2AF75980075A90C75A70F11
:10015E0075AB4375ADFB75AC1E75A71075C91875DB
:10016E00CA0075CB0075C80475A700758912758E07
:10017E0004758C00758A00C2A9D28C758D00758BA2
:10018E0000D2ABD28E75B62075D944C2992290009A
:10019E0093E09008A7F090009EE09008A8F09000E1
:1001AE009FE09008A9F09000BEE09008AAF09000A1
:1001BE00CBE09008ABF09000D9E09008ACF0900046
:1001CE00E7E09008ADF09000E9E09008AEF0900006
:1001DE00F7E09008AFF0900104E09008B0F09001C5
:1001EE0005E09008B1F0900117E09008B2F0900190
:1001FE002FE09008B4F090017DE09008B5F09001EA
:10020E007EE09008B6F090017FE09008B7F0900184
:10021E0016E09008B8F0900100E09008B9F0900058
:10022E00B7E09008BAF09000B8E09008BBF09000EC
:10023E00B2E09008BCF09000B3E09008BDF09001E1
:10024E001CE09008BEF090011DE09008BFF09001F8
:10025E001EE09008C0F090011FE09008C1F09001E0
:10026E0020E09008C2F09006D7E09008C3F0900608
:10027E00DBE09008C4F09006DFE09008C5F0900631
:10028E00E3E09008C6F09006E7E09008C7F090060D
:10029E00EBE09008C8F09006EFE09008C9F09006E9
:1002AE00F3E09008CAF09006F7E09008CBF09006C5
:1002BE00FBE09008CCF090077FE09008CDF090071F
:1002CE0080E09008CEF0900781E09008CFF0900784
:1002DE0082E09008D0F0900783E09008D1F090076C
:1002EE0084E09008D2F0900785E09008D3F0900754
:1002FE0086E09008D4F0900787E09008D5F090073C
:10030E0088E09008D6F0900789E09008D7F0900723
:10031E008AE09008D8F090078BE09008D9F090070B
:10032E008CE09008DAF090078DE09008DBF09007F3
:10033E008EE09008DCF090078FE09008DDF09001E1
:10034E0021E09008DEF0900122E09008DFF09001AD
:10035E0023E09008E0F0900124E09008E1F0900195
:10036E0025E09008E2F0900126E09008E3F090017D
:10037E0027E09008E4F0900128E09008E5F0900165
:10038E0029E09008E6F090012AE09008E7F022902C
:10039E0008A7E0900093F09008A8E090009EF090DF
:1003AE0008A9E090009FF09008AAE09000BEF0909F
:1003BE0008ABE09000CBF09008ACE09000D9F09044
:1003CE0008ADE09000E7F09008AEE09000E9F09004
:1003DE0008AFE09000F7F09008B0E0900104F090C4
:1003EE0008B1E0900105F09008B2E0900117F0908E
:1003FE0008B4E090012FF09008B8E0900116F0904C
:10040E0008B9E0900100F09008BAE09000B7F090C3
:10041E0008BBE09000B8F09008BCE09000B2F090FD
:10042E0008BDE09000B3F09008BEE090011CF09083
:10043E0008BFE090011DF09008C0E090011EF09002
:10044E0008C1E090011FF09008C2E0900120F090EA
:10045E0008C3E09006D7F09008C4E09006DBF09059
:10046E0008C5E09006DFF09008C6E09006E3F09035
:10047E0008C7E09006E7F09008C8E09006EBF09011
:10048E0008C9E09006EFF09008CAE09006F3F090ED
:10049E0008CBE09006F7F09008CCE09006FBF090C9
:1004AE0008CDE090077FF09008CEE0900780F090A6
:1004BE0008CFE0900781F09008D0E0900782F0908E
:1004CE0008D1E0900783F09008D2E0900784F09076
:1004DE0008D3E0900785F09008D4E0900786F0905E
:1004EE0008D5E0900787F09008D6E0900788F09046
:1004FE0008D7E0900789F09008D8E090078AF0902E
:10050E0008D9E090078BF09008DAE090078CF09015
:10051E0008DBE090078DF09008DCE090078EF090FD
:10052E0008DDE090078FF09008DEE0900121F0905A
:10053E0008DFE0900122F09008E0E0900123F090B7
:10054E0008E1E0900124F09008E2E0900125F0909F
:10055E0008E3E0900126F09008E4E0900127F09087
:10056E0008E5E0900128F09008E6E0900129F0906F
:10057E0008E7E090012AF02275480090089FE4F009
:10058E00A3F0753200753100754E00754F00C22C08
:10059E00D22D9008A8E06002D22474FE9008A1F833
:1005AE00E4F0E8A3F074FE9008A5F8E4F0E8A3F0F8
:1005BE0074FE9008A3F8E4F0E8A3F0745A9008F9DA
:1005CE00F0745A9008FAF0D22EC22AC230C22FC24C
:1005DE002BC232C23822750B00750A00AE0AAF0B61
:1005EE00AC08AD09EDC39FEC9E401674FF1272BFAE
:1005FE0075CF01780B740126F6500418E436F650C8
:10060E00DB22C2AF75D904758F0375B7A575B7F127
:10061E0090F800E4F0758F0175B7A575B7F1E52870
:10062E0090F800F075B7A575B7F190F801E4F07584
:10063E00B7A575B7F19008EDE090F802F075B7A583
:10064E0075B7F19008F1E090F803F075B7A575B79E
:10065E00F19008EEE090F804F075B7A575B7F1903B
:10066E0008EFE090F805F075B7A575B7F19008F0B2
:10067E00E090F806F075B7A575B7F19008F2E09026
:10068E00F807F0758F0075D944D2AF2290005BE069
:10069E00B4AB61C2AF75D90475B62275F522758FEC
:1006AE000375B7A575B7F1740090F600F0758F015C
:1006BE00755B00755A00AE5AAF5B7445BE00279F3E
:1006CE00402475B7A575B7F19008A7120048E0FC55
:1006DE0090F600120048ECF0785B740126F6500498
:1006EE0018E436F650D0758F0075F51175B6207575
:1006FE00D944D2AF22C2AF75F52275D904755B000D
:10070E00755A00AE5AAF5B7445BE00229F401F90D3
:10071E00F600120048E493FC9008A7120048ECF093
:10072E00785B740126F6500418E436F650D575D968
:10073E004475F511D2AF2290005BE0B4AA0280039B
:10074E00020882C2AF75D90475B62275F522758F6F
:10075E000375B7A575B7F1740090F400F075B7A5E1
:10076E0075B7F1740090F200F075B7A575B7F17416
:10077E000090F000F075B7A575B7F1740090EE001B
:10078E00F0758F01755B00755A00AE5AAF5B74FF42
:10079E00C39F74019E402475B7A575B7F190009163
:1007AE00120048E0FC90F400120048ECF0785B7404
:1007BE000126F6500418E436F650CF755B00755AD4
:1007CE0000AE5AAF5B74FFC39F74019E402475B791
:1007DE00A575B7F1900291120048E0FC90F200125C
:1007EE000048ECF0785B740126F6500418E436F6F7
:1007FE0050CF755B00755A00AE5AAF5B74FFC39F46
:10080E0074019E402475B7A575B7F190049112003E
:10081E0048E0FC90F000120048ECF0785B74012682
:10082E00F6500418E436F650CF755B00755A00AEDC
:10083E005AAF5B74FFC39F74019E402475B7A575B4
:10084E00B7F1900691120048E0FC90EE00120048BD
:10085E00ECF0785B740126F6500418E436F650CFAF
:10086E00758F0075F51175B62075D944D2AF743AEF
:10087E00900791F02290005BE0B4AA028003020977
:10088E00C0C2AF75D90475B62275F522758F037582
:10089E00B7A575B7F1740090EC00F075B7A575B7F4
:1008AE00F1740090EA00F075B7A575B7F174009079
:1008BE00E800F075B7A575B7F1740090E600F07515
:1008CE008F01755B00755A00AE5AAF5B74FFC39F04
:1008DE0074019E402475B7A575B7F1900091120072
:1008EE0048E0FC90EC00120048ECF0785B740126B6
:1008FE00F6500418E436F650CF755B00755A00AE0C
:10090E005AAF5B74FFC39F74019E402475B7A575E3
:10091E00B7F1900291120048E0FC90EA00120048F4
:10092E00ECF0785B740126F6500418E436F650CFDE
:10093E00755B00755A00AE5AAF5B74FFC39F7401AE
:10094E009E402475B7A575B7F1900491120048E04A
:10095E00FC90E800120048ECF0785B740126F6502B
:10096E000418E436F650CF755B00755A00AE5AAFD8
:10097E005B74FFC39F74019E402475B7A575B7F1D4
:10098E00900691120048E0FC90E600120048ECF050
:10099E00785B740126F6500418E436F650CF758F46
:1009AE000075F51175B62075D944D2AF743A90071B
:1009BE0091F022C2AF75D90475F522755B00755A98
:1009CE0000AE5AAF5B74FFC39F74019E401F90F43C
:1009DE0000120048E493FC900091120048ECF0786D
:1009EE005B740126F6500418E436F650D4755B009D
:1009FE00755A00AE5AAF5B74FFC39F74019E401FC1
:100A0E0090F200120048E493FC900291120048EC20
:100A1E00F0785B740126F6500418E436F650D4755F
:100A2E005B00755A00AE5AAF5B74FFC39F74019E94
:100A3E00401F90F000120048E493FC9004911200C5
:100A4E0048ECF0785B740126F6500418E436F65044
:100A5E00D4755B00755A00AE5AAF5B74FFC39F74BA
:100A6E00019E401F90EE00120048E493FC90069108
:100A7E00120048ECF0785B740126F6500418E43648
:100A8E00F650D475F51175D944D2AF74019000DAD1
:100A9E00F0743A900791F09009007401F022C2AF01
:100AAE0075D90475F522755B00755A00AE5AAF5BA9
:100ABE0074FFC39F74019E401F90EC00120048E427
:100ACE0093FC900091120048ECF0785B740126F6CE
:100ADE00500418E436F650D4755B00755A00AE5AC1
:100AEE00AF5B74FFC39F74019E401F90EA0012001B
:100AFE0048E493FC900291120048ECF0785B74018C
:100B0E0026F6500418E436F650D4755B00755A007C
:100B1E00AE5AAF5B74FFC39F74019E401F90E800F6
:100B2E00120048E493FC900491120048ECF0785BBC
:100B3E00740126F6500418E436F650D4755B007531
:100B4E005A00AE5AAF5B74FFC39F74019E401F9054
:100B5E00E600120048E493FC900691120048ECF077
:100B6E00785B740126F6500418E436F650D475F509
:100B7E001175D944D2AF74029000DAF0743A90072E
:100B8E0091F07402900900F02274019000DAF09056
:100B9E0008A8E0903C1EF828287380188016A2A39F
:100BAE00400674029000DAF0800AA2A44006740295
:040BBE009000DAF0D9
:0C3C1E00020BA8020BAA020BAC020BB8B0
:100BC2009000DAE0B40105A236B34002801AD236B0
:100BD2001247191209C174019000DAF012039D1232
:100BE2003EC0741B90005FF09000DAE0B40206A2EF
:100BF20036B3B34002801AC236124719120AAC74D5
:100C0200029000DAF012039D123EC0741B90005F46
:100C1200F022E54F64046006E59964FF60028031CA
:100C2200A22C4004D22C8027E54F600874E6254FA1
:100C320090005FF0E54E600874F0254E90005FF082
:100C4200E54FB4010280FE754F00754E00C22C8044
:100C520002C22CE54F903C2AF8282873754F00E514
:100C620099B4FF03754E01E599B4FE03754E02E592
:100C720099B4FD03754E03E599B4FC03754E04E582
:100C820099B4FA03754E05E599B4FB06754F011246
:100C92004719E599B4F906754F04124719E599B455
:100CA200F733124719C29C74AB90005BF012069A9C
:100CB20074AA90005BF0900900E0B40105120745A8
:100CC200800312088390005BE4F0D29C754F00759C
:100CD2004E007599F7E599D394E54007E599C394D9
:100CE200F040028016859950754F027E017F00E523
:100CF20050C394E61272DF8E338F3490089FE4F073
:100D0200A3F0E599D394C24007E599C394E6400263
:100D12008028859950754F0374E5C39550F5347555
:100D22003300AE33AF34906C601272AEE493F87459
:100D3200019390089FC8F0A3C8F0D2990210A29024
:100D420008B4E0700AA225B35005A226B34002807F
:100D52005C90089FE0FEA3E0FF74FFBE00039F507B
:100D620009EFC39446EE9406402B90089FE0FEA341
:100D7200E0FFEFD3946DEE94064009EFC394EEEEDC
:100D82009406401190089FE0FEA3E0FFEFD394FF8A
:100D9200EE9406401390089FE0FEA3E0FF900091BE
:100DA200120048E599F08003859975801190089F9B
:100DB200E0FEA3E0FF900091120048E599F0900850
:100DC2009F1272ED90089FE0FEA3E0FFEFB40106D0
:100DD200EEB407028003020E9B900791E0B43C023E
:100DE2008003020E9BA225B35005A226B3400280C7
:100DF20055C29C12039D90009EE09008FFF01240A5
:100E02000790017DE09008B5F090017EE09008B671
:100E1200F090017FE09008B7F074AB90005BF012A5
:100E2200069A74AA90005BF0900900E0B4010512E2
:100E320007458003120883900900E09000DAF090E1
:100E4200005BE4F08048C29C12019C74009008B5DB
:100E5200F074009008B6F074009008B7F090009E0D
:100E6200E09008FFF012400774AB90005BF01206AE
:100E72009A74AA90005BF0120745120883D29C75FF
:100E820099FB7464F5097508001205E480FED29C92
:100E9200754F00754E007599FB0210A290089FE0F5
:100EA200FEA3E0FFEF4E700685993275310090087F
:100EB2009FE0FEA3E0FF74016F4E701BAC31AD32B8
:100EC200AA33AB34ED2BFBEC3AFA8A068B0790007F
:100ED20091120048E599F090089F1272ED90089FD8
:100EE200E0FEA3E0FF74026F4E7021AC31AD3274AC
:100EF200566D4C7006E55064E66002800312471995
:100F0200124007855099754F00754E000210A2904D
:100F1200089FE0FEA3E0FF900091120048E599F0DF
:100F220090089F1272ED90089FE0FEA3E0FFAC33A1
:100F3200AD348F028E038C068D07906CA61272AEB2
:100F4200E493F9740193FEEAD39EEB99400985502C
:100F520099754F00754E000210A290089FE0FEA303
:100F6200E0FF900091120048E599F090089F1272FC
:100F7200ED90089FE0FEA3E0FFEFB40006EEB4019F
:100F82000280030210A2900071E0D394C7400B903C
:100F92000071E0C394C8F551801A900071E0D394B7
:100FA20063400B900071E0C39464F5518006900099
:100FB20071E0F551E55175F002A4FFAEF08F74EFC8
:100FC200900091127310EFFCE0FDEC90009412730C
:100FD20010EDFCE0FDEC2DB5510280030210930FE1
:100FE200EF900091127310E574FFE0FCEF90009512
:100FF200127310ECFFE0FCEFC39CB55102800302B8
:101002001093E574900093127310E574FFE0FCEF07
:10101200900096127310ECFFE0FCEF2CB55172E5D4
:1010220074900097127310E0C395519008EDF0E5AB
:1010320074900098127310E0C395519008EEF0E599
:101042007490009B127310E0C395519008EFF0E585
:101052007490009C127310E0C395519008F0F0E573
:101062007490009D127310E0C395519008F1F0E561
:101072007490009E127310E0C395519008F2F01222
:1010820006107599F97464F5097508001205E48073
:10109200FE7599FF7464F5097508001205E480FE77
:0F3C2A00020C5E020D41020E9E020F11020F5C92
:1010A20022E54E903C39F828287302118790089F58
:1010B200E0FEA3E0FF900061120048E0F59990087D
:1010C2009F1272ED90089FE0FEA3E0FF741C6F4E2A
:1010D2007003754E00021187856F9902118790087F
:1010E2009FE0FEA3E0FF900091120048E0F599EF27
:1010F200B40107EEB40703754E0090089F1272ED1B
:071102000211879008A0E034
:0F3C39000210AC0210AF0210DA0210E002110507
:10110900903CABF82828738553998067856099804E
:1011190062856299805D8566998058856899805352
:10112900856999804E856A998049856B9980449033
:10113900001FE0F599803CA22DB340077599FAC2CA
:101149002D8017A224B3400575990F800B90005F7D
:10115900E0F59990005FE4F0C2248017856C9980CE
:1011690012856799800D856D9980087599FC8003B2
:03117900754E00B0
:103CAB0002111002111502111A02111F0211240226
:103CBB00112902112E021133021138021140021187
:0D3CCB006502116A02116F02117402117975
:0B117C0090089F1272ED8003123F1BD1
:033C4800021184E2
:1011870022E538255BFFAE5A50010E900091120000
:1011970048E0F539E538255BFFAE5A50010E0FBF21
:1011A70000010E900091120048E0F53A85403CE5B9
:1011B70039B53A058539388041E53AD39539401D27
:1011C700E53AC39539853BF0A4FFAEF0E53C8E04C4
:1011D7008F05FF1272CFED2539F538801DE539C32C
:1011E700953A853BF0A4FFAEF0E53C8E048F05FFF2
:1011F7001272CFEDF4042539F53822E53AD3953943
:10120700401DE53AC39539853BF0A4FFAEF0E53CB8
:101217008E048F05FF1272CFED2539F538801DE555
:1012270039C3953A853BF0A4FFAEF0E53C8E048FB9
:1012370005FF1272CFEDF4042539F5382290009797
:10124700E0B4017FE56875F00A84FF7E008F38E51A
:101257006875F00A84ADF07C008D3B75400A755ABD
:1012670005755B24E538C394115005121188800673
:101277009005C6E0F538E538C394F05008E5389096
:101287000083F0800674EF900083F0E56875F00A3C
:1012970084FF7E008F38E56875F00A84ADF07C0026
:1012A7008D3B75400A755A05755B5AE538C394112D
:1012B700500512118880069005FCE0F538E5389056
:1012C700005AF022900097E0B401028003021359FC
:1012D700E56875F00A84FF7E008F38E56875F00AC7
:1012E70084ADF07C008D3B75400A755A05755B36F9
:1012F700E538C39411500512118880069005D8E08F
:10130700F538E538C394F0500585384C8003754CA3
:10131700EFE56875F00A84FF7E008F38E56875F0A1
:101327000A84ADF07C008D3B75400A755A05755BE4
:1013370048E538C39411500512118880069005EAD4
:10134700E0F538E538C394F0500585384D800375CE
:101357004DEF22E56075F00484FF7E008F38E5606D
:1013670075F00484ADF07C008D3B754004755A011F
:10137700755B00E538C3943F5005121188800690CD
:1013870001D0E0F538E538900899F8E4F0E8A3F0E3
:1013970090005EE075F020A4FFAEF09000E2E08ED2
:1013A700048F05FF1272CF8D389000CAE0D3956085
:1013B70050030214659000EEE0D395604010ED9065
:1013C70001D1127310E0F52C752B00021462900006
:1013D700B9E0D395604043E5389001D1127310E02E
:1013E700F539E5389001F1127310E0F53A9000EE07
:1013F700E0F4042560F53B9000B9E0FE9000EEE0D4
:10140700F4042EF53CE539B53A05853938800312E1
:10141700120285382C752B008041E5389001F112B6
:101427007310E0F539E538900211127310E0F53AC0
:101437009000B9E0F4042560F53B9000CAE0FE9007
:1014470000B9E0F4042EF53CE539B53A058539389D
:10145700800312120285382C752B0002150C9000A0
:10146700F1E0D395605011E538900251127310E006
:10147700F52C752B0002150C9000BAE0D39560503F
:1014870043E538900231127310E0F539E5389002E0
:1014970051127310E0F53A9000BAE0F4042560F5B4
:1014A7003B9000F1E0FE9000BAE0F4042EF53CE535
:1014B70039B53A05853938800312120285382C75FB
:1014C7002B008041E538900211127310E0F539E5E1
:1014D70038900231127310E0F53A9000CAE0F40434
:1014E7002560F53B9000BAE0FE9000CAE0F4042EB8
:1014F700F53CE539B53A058539388003121202857E
:10150700382C752B0022900102E0F53D75401175CE
:101517005A02755B00AE52AF53E53D75F00FA4FD5F
:10152700ACF0EDD39FEC9E4021E53D8E048F05FF87
:101537001272CFED75F010A4FFAEF0E56075F011F3
:1015470084FD7C00ED2FF53E800EE56075F011847B
:10155700FF7E00EF24F0F53E853E38E56075F0111B
:1015670084AFF07E008F3B12118885383FAE52AFB3
:1015770053900102E075F00FA4FDACF0EDD39FECA2
:101587009E4028755A02755B10853E381211888572
:101597003F3985383AAE52AF53E53D8E048F05FF8C
:1015A7001272FA8D3B853D3C121202E5389008997C
:1015B700F8E4F0E8A3F0752C64752B002290010283
:1015C700E0F53D754011755A02755B00AE52AF5399
:1015D700E53D75F00FA4FDACF0EDD39FEC9E4021E7
:1015E700E53D8E048F05FF1272CFED75F010A4FF55
:1015F700AEF0E56275F01184FD7C00ED2FF53E80BD
:101607000EE56275F01184FF7E00EF24F0F53E854C
:101617003E38E56275F01184AFF07E008F3B121102
:101627008885383FAE52AF53900102E075F00FA4A2
:10163700FDACF0EDD39FEC9E4028755A02755B1008
:10164700853E38121188853F3985383AAE52AF53F7
:10165700E53D8E048F05FF1272FA8D3B853D3C12E6
:101667001202E538900899F8E4F0E8A3F0E56C6019
:1016770017E56CC394FE50109000F6E0B402099091
:1016870000E4E0D3940B5002801F900899E0FEA37A
:10169700E0FFE56C1272DF74E78E048F05FF1272AC
:1016A700CF900899ECF0A3EDF09000CCE0B4045F84
:1016B700E56075F00484FF7E008F38E56075F004FF
:1016C70084ADF07C008D3B754004755A01755B0055
:1016D700E538C3943F500512118880069001D0E089
:1016E700F538900899E0FEA3E0FFE5381272DF7441
:1016F700328E048F05FF1272CF900899E0FEA3E0A7
:10170700FFEF2DFDEE3CFC900899ECF0A3EDF07592
:101717002C64752B0022900097E0B40146E56875AC
:10172700F00A84FF7E008F38E56875F00A84ADF013
:101737007C008D3B75400A755A05755B00E538C31B
:101747009411500512118880069005A2E0F538AE75
:101757002BAF2CE5382FFF50010E74641273228EC5
:101767002B8F2C900098E0B40146E56975F00A8448
:10177700FF7E008F38E56975F00A84ADF07C008D37
:101787003B75400A755A05755B6CE538C394115073
:1017970005121188800690060EE0F538AE2BAF2CA7
:1017A700E5382FFF50010E74641273228E2B8F2C95
:1017B7009000A7E0B40249E56BC3944175F0058436
:1017C700FF7E008F38E56B75F00584ADF07C008DEA
:1017D7003B754005755A06755B00E538C394135091
:1017E7000512118880069006A4E0F538AE2BAF2CC1
:1017F700E5382FFF50010E74641273228E2B8F2C45
:101807009000E9E0B4020280030218BCE56075F0BD
:101817001584FF7E008F38E56075F01584ADF07C88
:10182700008D3B754015755A03755BF4E538C39415
:101837000B50051211888006900490E0F538E538C2
:1018470075F0FFA4FFAEF09000EAE08E048F05FF6D
:101857001272CFED90007FF0E56775F078A4FFAEC8
:10186700F074FF8E048F05FF1272CF8C5A8D5B7454
:10187700028C068D071200398F38AC5AAD5B7404A1
:10188700FF1272FA8D3B754004755A06755B28E5A1
:1018970038C3941D500512118880069006D6E0F5CE
:1018A70038AE2BAF2CE5382FFF50010E746412733E
:1018B700228E2B8F2C900096E0B4025DE56275F0C6
:1018C70064A4FFAEF074081200398E5C8F5D740556
:1018D7008E048F05FF1272CF8D38AE5CAF5D740535
:1018E7008E048F05FF1272FA8D3B754005755A05F8
:1018F700755BDEE538C39413500512118880069096
:101907000682E0F538AE2BAF2CE5382FFF50010EDD
:1019170074641273228E2B8F2C9000D8E0707F9006
:10192700005EE075F00A84FF7E008F3890005EE06D
:1019370075F00A84ADF07C008D3B75400A755A0539
:10194700755BC0E538C3940E500512118880069068
:10195700065FE0F538E538900084F09000F7E0B4D2
:10196700023C90005EE075F00A84FF7E008F38909D
:10197700005EE075F00A84ADF07C008D3B75400A8F
:10198700755A05755BCFE538C3940E50051211885B
:10199700800690066EE0F538E538900085F02290D5
:1019A700009FE0B401179008F4E0252CFFAE2B5000
:1019B700010E9000F3E01273228E2B8F2C900117EB
:1019C700E0B40114900118E0A852B80004955350F0
:1019D70007E560C39561400280139000C1E0252CA4
:1019E700FFAE2B50010E8E2B8F2C021E0D90009FE9
:1019F700E0B40306A22AB3B3400280509008FEE089
:101A070070109008F7E0C39405A852B800069553E4
:101A1700400280109000C1E0252CFFAE2B50010E34
:101A27008E2B8F2C9008FEE0600D9008F7E0A852EF
:101A3700B800069553400280109000C1E0252CFFA6
:101A4700AE2B50010E8E2B8F2C021E0D900099E0AD
:101A5700B402028003021E0D90009CE0602FE5682F
:101A6700D394464028900016E0FEA3E0FF9000D7ED
:101A7700E075F003A4FDACF0EFD39DEE9C400E9013
:101A870000FBE0A852B80005D395535003021E0D82
:101A97009000CCE0B403028003021C5585625B759D
:101AA7005A009000A3E0A852B800049553500E9036
:101AB70000A4E0A85AB80005D3955B5003021C5256
:101AC700E56275F002A4FFAEF074158E048F05FF72
:101AD7001272CF8C068D07900621120048FEE0FF98
:101AE700EE90009BE0FEEF8E0088F0A4FFAEF0744E
:101AF700648E048F05FF1272CF8C5A8D5B90005E47
:101B0700E075F018A4FFAEF09000E2E08E048F05B8
:101B1700FF1272CF8C068D07900639120048AE5A15
:101B2700AF5BE01272DF74648E048F05FF1272CF11
:101B37008C5A8D5BE566A85AB80005D3955B5003B0
:101B4700021BC9E566C3955BFFE4955AFE8E5A8F63
:101B57005B7428BE00039F500C755B28755A007490
:101B67000D90005FF0AE5AAF5B90009CE01272DF01
:101B770074288E048F05FF1272CF8C5A8D5B9008E4
:101B870099E0FEA3E0FF740A8E048F05FF1272CF5F
:101B97008D068C07AC5AAD5BCFCECF120003740A0B
:101BA7008E048F05FF1272CF8C5A8D5B900899E0D7
:101BB700FEA3E0FF12732A900899EEF0A3EFF0025C
:101BC7001C52E566A85AB80004955B507EAE5AAF22
:101BD7005BE5661273228E5A8F5B7428BE00039FE3
:101BE700500C755B28755A00740D90005FF0AE5A63
:101BF700AF5B90009CE01272DF74288E048F05FFA4
:101C07001272CF8C5A8D5B900899E0FEA3E0FF74A7
:101C17000A8E048F05FF1272CF8D068C07AC5AAD62
:101C27005BCFCECF120003740A8E048F05FF1272AA
:101C3700CF8C5A8D5B900899E0FEA3E0FFEF2DFD56
:101C4700EE3CFC900899ECF0A3EDF0021E0D90001D
:101C5700E4E08560F0A4FFAEF074051272DF74074C
:101C67001200398E5A8F5B9000A3E0A852B8000487
:101C7700955350129000A4E075F002A4FDACF0EF6C
:101C8700C39DEE9C4003021E0DE56075F00B84FFBB
:101C97007E00900621120048FEE0FFEE90009BE0D8
:101CA700FEEF8E0088F0A4FFAEF074648E048F05FB
:101CB700FF1272CF8C5A8D5B90005EE075F018A40E
:101CC700FFAEF09000E2E08E048F05FF1272CF8C1A
:101CD700068D07900639120048AE5AAF5BE01272C4
:101CE700DF74648E048F05FF1272CF8C5A8D5BE50B
:101CF70066A85AB80005D3955B5003021D84E566B4
:101D0700C3955BFFE4955AFE8E5A8F5B7428BE001D
:101D1700039F500C755B28755A00740D90005FF097
:101D2700AE5AAF5B90009CE01272DF74288E048F6E
:101D370005FF1272CF8C5A8D5B900899E0FEA3E0E5
:101D4700FF740A8E048F05FF1272CF8D068C07ACC5
:101D57005AAD5BCFCECF120003740A8E048F05FFF6
:101D67001272CF8C5A8D5B900899E0FEA3E0FF12A8
:101D7700732A900899EEF0A3EFF0021E0DE566A80E
:101D87005AB80004955B507EAE5AAF5BE566127396
:101D9700228E5A8F5B7428BE00039F500C755B28F8
:101DA700755A00740D90005FF0AE5AAF5B90009CBF
:101DB700E01272DF74288E048F05FF1272CF8C5ADF
:101DC7008D5B900899E0FEA3E0FF740A8E048F05EF
:101DD700FF1272CF8D068C07AC5AAD5BCFCECF12F8
:101DE7000003740A8E048F05FF1272CF8C5A8D5B25
:101DF700900899E0FEA3E0FFEF2DFDEE3CFC900874
:101E070099ECF0A3EDF0229000F7E0B4027BE560D7
:101E170075F00884FF7E008F38E56075F00884ADA3
:101E2700F07C008D3B754008755A01755BE0E5381D
:101E3700C3943F50051211888006900290E0F53850
:101E4700E53890089BF8E4F0E8A3F090089BE0FEE3
:101E5700A3E0FFAC2BAD2C12000374648E048F0536
:101E6700FF1272CF90089BECF0A3EDF0900094E086
:101E77008C068D071272DF74648E048F05FF127251
:101E8700CF90089BECF0A3EDF0900899E0FEA3E05B
:101E9700FFAC2BAD2C12000374648E048F05FF1268
:101EA70072CF900899ECF0A3EDF0900094E08C06C7
:101EB7008D071272DF74648E048F05FF1272CF9044
:101EC7000899ECF0A3EDF0A204401DAE52AF537495
:101ED70005BE00039F5002D204E562D394CC4008AC
:101EE700D202741190005FF0229000F6E0B402086D
:101EF7009000E4E0640B60028045900899E0FEA33F
:101F0700E0FFE56C1272DF74E78E048F05FF127233
:101F1700CF900899ECF0A3EDF09000F7E0B4021F22
:101F270090089BE0FEA3E0FFE56C1272DF74E78E7A
:101F3700048F05FF1272CF90089BECF0A3EDF09091
:101F470000B6E05402601B9000ADE0A852B8001242
:101F5700D39553400DA204B3B35007E562C3949AD7
:101F67004002805FAE35AF369000ABE075F002A45B
:101F7700FDACF0EF2DFDEE3CFC74022DFD50010C85
:101F8700E562BC003ED39D403A754401A23140331F
:101F97009000ACE075F05EA4FDACF07405FF127222
:101FA700CF8C5C8D5D124A9C900899E0FEA3E0FF00
:101FB7009000ACE02FFF50010E900899EEF0A3EFD0
:101FC700F0D231E562A835B8000495365002C23127
:101FD700856236753500E54470030220E6900109F5
:101FE700E0C3954450030220D8900119E0C394023E
:101FF7004003022082E56875F00A84FF7E009005A1
:1020070091120048E0F55B755A00AE5AAF5B90003D
:10201700ACE01272DF74648E048F05FF1272CF8CEE
:102027005C8D5D900109E004C395448C068D071211
:1020370072DF900109E08E048F05FF1272CF8C5C6E
:102047008D5D900899E0FEA3E0FFEF2DFDEE3CFCCF
:10205700900899ECF0A3EDF09000F7E0B4021A9025
:10206700089BE0FEA3E0FFAA5CAB5DEF2BFBEE3A1B
:10207700FA90089BEAF0A3EBF08056900109E00480
:10208700C39544854CF0A4FFAEF0900109E08E049F
:102097008F05FF1272CF8C5C8D5D900899E0FEA3CF
:1020A700E0FFEF2DFDEE3CFC900899ECF0A3EDF07E
:1020B7009000F7E0B4021A90089BE0FEA3E0FFAAA5
:1020C7005CAB5DEF2BFBEE3AFA90089BEAF0A3EBD3
:1020D700F00544900109E0C395445003754400900E
:1020E70000B6E05401601B9000AAE0A852B80012A5
:1020F700D39553400DA204B3B35007E560C394CC06
:10210700400280609000A8E075F003A4FFAEF0E500
:10211700412FFF50010E74032FFF50010EE560BEE3
:102127000042D39F403E754501A23140379000A938
:10213700E075F05EA4FFAEF074058E048F05FF1204
:1021470072CF8C5C8D5D124A9C900899E0FEA3E0EB
:10215700FF9000A9E02FFF50010E900899EEF0A321
:10216700EFF0D231E560C395415002C2318560413D
:10217700E545700302228090010AE0C395455003AC
:10218700022272900119E0C39402400302221CE567
:102197006875F00A84FF7E00900591120048E0F50B
:1021A7005B755A00AE5AAF5B9000A9E01272DF74FC
:1021B700648E048F05FF1272CF8C5C8D5D90010ACF
:1021C700E004C395458C068D071272DF90010AE083
:1021D7008E048F05FF1272CF8C5C8D5D900899E09D
:1021E700FEA3E0FFEF2DFDEE3CFC900899ECF0A379
:1021F700EDF09000F7E0B4021A90089BE0FEA3E030
:10220700FFAA5CAB5DEF2BFBEE3AFA90089BEAF076
:10221700A3EBF0805690010AE004C39545854DF085
:10222700A4FFAEF090010AE08E048F05FF1272CF73
:102237008C5C8D5D900899E0FEA3E0FFEF2DFDEE2D
:102247003CFC900899ECF0A3EDF09000F7E0B402A5
:102257001A90089BE0FEA3E0FFAA5CAB5DEF2BFBA7
:10226700EE3AFA90089BEAF0A3EBF0054590010AD5
:10227700E0C395455003754500900899E0FEA3E03B
:10228700FF9000BBE0BE00039F500D9000BBE090A5
:102297000899F8E4F0E8A3F09000F7E0B402129090
:1022A700089BE0FEA3E0FF9000BBE0BE00059F4057
:1022B70002800D9000BBE090089BF8E4F0E8A3F0E3
:1022C700229000F7E0B401028003022416A204B3AF
:1022D70050030223FD9000C2E0B4017A900899E010
:1022E700FEA3E0FFAC52AD53120003743C8E048F83
:1022F70005FF1272CF9000D2E0BC00159D401290EE
:102307000899E0FEA3E0FF9000D4E0BE00039F50D1
:1023170002D203900899E0FEA3E0FFAC52AD53123E
:102327000003743C8E048F05FF1272CF9000D2E039
:10233700C3940ABC001AD39D4016900899E0FEA3E7
:10234700E0FF9000D4E0C39405BE0004D39F500281
:102357008002C203807A900899E0FEA3E0FFAC52A6
:10236700AD5312000374788E048F05FF1272CF905D
:1023770000D2E0BC00159D4012900899E0FEA3E052
:10238700FF9000D4E0BE00039F5004D20380419029
:102397000899E0FEA3E0FFAC52AD53120003747836
:1023A7008E048F05FF1272CF9000D2E0C3940ABC4F
:1023B700001AD39D4016900899E0FEA3E0FF900015
:1023C700D4E0C39405BE0004D39F50028002C20329
:1023D700A203B34021900899E0FEA3E0FF9000D349
:1023E700E01272DF74648E048F05FF1272CF9008BB
:1023F70099ECF0A3EDF0A203B3400CA235400674AC
:102407002490005FF0D235A2034002C2358002C299
:102417000390005AE06006A204B3B340028019900B
:102427000899E0FEA3E0FF90005AE02FFF50010E4D
:10243700900899EEF0A3EFF0A201B34006A202B311
:10244700B3500990001EE4F0A3F0802D900899E0A6
:10245700FEA3E0FF7400D39F74019E40119008997A
:10246700E0F8A3E090001EC8F0A3C8F0800B74FF4B
:1024770090001EF8E4F0E8A3F09000D9E0C39404BC
:10248700400C9008FBE0C3940240030225709000C3
:10249700C2E0B40147900899E0FEA3E0FF745E1222
:1024A70072DF74058E048F05FF1272CF900899ECC6
:1024B700F0A3EDF09000F7E0B4021F90089BE0FE58
:1024C700A3E0FF745E1272DF74058E048F05FF129E
:1024D70072CF90089BECF0A3EDF08045900899E04F
:1024E700FEA3E0FF745E1272DF740A8E048F05FF8D
:1024F7001272CF900899ECF0A3EDF09000F7E0B4DA
:10250700021F90089BE0FEA3E0FF745E1272DF7467
:102517000A8E048F05FF1272CF90089BECF0A3ED93
:10252700F0900899E0FEA3E0FF7402BE000CD39F71
:102537004008752A02752900800A900899E0F52954
:10254700A3E0F52A90089BE0FEA3E0FF7402BE001B
:102557000CD39F4008752E02752D00800A90089BAA
:10256700E0F52DA3E0F52E8046900899E0FEA3E064
:10257700FF7401BE000CD39F4008752A017529001E
:10258700800A900899E0F529A3E0F52A90089BE0D6
:10259700FEA3E0FF7401BE000CD39F4008752E0117
:1025A700752D00800A90089BE0F52DA3E0F52E908D
:1025B700001CE529F0A3E52AF0A238B34009C201BF
:1025C70090001EE4F0A3F02290005EE090039112C9
:1025D7007310E0F54275436490005EE0FE9000CD15
:1025E700E0D39E4037E56075F00884FF7E008F38A2
:1025F700E56075F00884ADF07C008D3B754008758B
:102607005A03755B96E538C3941F500512118880ED
:1026170006900446E0F5388538438035E56075F067
:102627000884FF7E008F38E56075F00884ADF07C84
:10263700008D3B754008755A03755BB6E538C39442
:102647001F50051211888006900466E0F53885381A
:102657004322900103E0F53D754011755A04755BFF
:1026670000AE52AF53E53D75F00FA4FDACF0EDD3CE
:102677009FEC9E4021E53D8E048F05FF1272CFED42
:1026870075F010A4FFAEF0E56075F01184FD7C00D5
:10269700ED2FF53E800EE56075F01184FF7E00EFAB
:1026A70024F0F53E853E38E56075F01184AFF07E85
:1026B700008F3B12118885383FAE52AF539001030C
:1026C700E075F00FA4FDACF0EDD39FEC9E402875AC
:1026D7005A04755B10853E38121188853F39853855
:1026E7003AAE52AF53E53D8E048F05FF1272FA8D55
:1026F7003B853D3C121202853842754364229001A6
:1027070003E0F53D754011755A04755B00AE52AF95
:1027170053E53D75F00FA4FDACF0EDD39FEC9E4063
:1027270021E53D8E048F05FF1272CFED75F010A4E1
:10273700FFAEF0E56275F01184FD7C00ED2FF53EEC
:10274700800EE56275F01184FF7E00EF24F0F53E00
:10275700853E38E56275F01184AFF07E008F3B123D
:10276700118885383FAE52AF53900103E075F00FE3
:10277700A4FDACF0EDD39FEC9E4028755A04755B21
:1027870010853E38121188853F3985383AAE52AFE9
:1027970053E53D8E048F05FF1272FA8D3B853D3C54
:1027A7001212028538427543649000FEE0B4047942
:1027B70090005EE0FE9000CDE0D39E4037E5607567
:1027C700F00884FF7E008F38E56075F00884ADF06F
:1027D7007C008D3B754008755A03755B96E538C3D9
:1027E700941F50051211888006900446E0F538853D
:1027F70038438035E56075F00884FF7E008F38E543
:102807006075F00884ADF07C008D3B754008755A03
:1028170003755BB6E538C3941F500512118880060F
:10282700900466E0F53885384322900097E0B401BC
:102837003BE56875F00A84FF7E008F38E56875F020
:102847000A84ADF07C008D3B75400A755A05755BAF
:1028570012E538C39411500512118880069005B40B
:10286700E0F538E5432538C39464F543900098E0D4
:10287700B4013BE56975F00A84FF7E008F38E5698E
:1028870075F00A84ADF07C008D3B75400A755A05DA
:10289700755B7EE538C39411500512118880069048
:1028A7000620E0F538E5432538C39464F543E5424F
:1028B7002543F53790009FE0B402109008F3E02518
:1028C70037FE9000F3E0F4042EF5379000F6E0D3DE
:1028D70094014040E56CC394E7501D74E7C3956CC1
:1028E700FE9008F5E08E00F5F0E884FF7E008F3853
:1028F700E5372538F537801CE56CC394E7FE90086B
:10290700F5E08E00F5F0E884FF7E008F38E537C3E9
:102917009538F537A2044006E5422464F537E537D4
:10292700D394644009E537C39464F537800375375A
:10293700009000CFE0C3953750069000CFE0F53701
:1029470022D201900082E0A852B800049553503E6D
:10295700900082E0A852B800049553500375370FD2
:10296700900082E004A852B80004955350037537CD
:1029770007900082E02402A852B800049553500241
:10298700C201900082E06006740990005FF0C230D7
:102997007E017F009000D5E01272DF9000E4E08EA8
:1029A700048F05FF1272CFE560BC000CD39D400871
:1029B700D238740A90005FF0900097E0B401099054
:1029C70000D6E0C39568400280159000E8E0A85261
:1029D700B8000495535002C201740B90005FF09049
:1029E7000097E0B40107E568C394644002801D9036
:1029F700012EE0600D90012EE0A852B80006955315
:102A070040028008C201740B90005FF0A2014003EE
:102A1700753700C237900117E0B40114900118E030
:102A2700A852B8000495535007E560C3956140026A
:102A3700802A9000C0E0D3941D400B9000C0E0C3F3
:102A4700941EF5378003753700A23440087415903B
:102A5700005FF0D237D234D232022B42C232C234B4
:102A670090009FE0B40306A22AB3B34003022B42AF
:102A77009008F7E0C39405A852B800049553500690
:102A87009008FEE06002801F9000C0E0D3941D40D4
:102A97000B9000C0E0C3941EF537800375370074B0
:102AA7000C90005FF0D2379008F7E0A852B8000406
:102AB700955350069008FEE07002801F9000C0E01A
:102AC700D3941D400B9000C0E0C3941EF5378003DC
:102AD700753700740C90005FF0D2379008F7E0A8C4
:102AE70052B80004955350319000DEE0B40228D26A
:102AF700309008FDE0FE9008FEE0D39E5006900857
:102B0700FEE0700280099008FDE4F0C23080069074
:102B170008FDE004F08002C2019008F7E02405A850
:102B270052B80004955350139000DEE0B4020A90A7
:102B370008FEE07002D2308002C201A22FB3402704
:102B47009000C0E0D3941D400B9000C0E0C3941EDA
:102B5700F5378003753700A2334006741090005F85
:102B6700F0D233D2378002C23385376D9000C0E090
:102B7700D3941D401890008EE02537FE90005EE04C
:102B870075F01E84FC7F00EE2CF5378029A237B341
:102B9700400890008EE0F537801C900090E02537C4
:102BA700FE90008EE02EFE90005EE075F01E84FC25
:102BB7007F00EE2CF537A238B34005D230756D0093
:102BC7002290005EE075F00584FF7E008F3890004C
:102BD7005EE075F00584ADF07C008D3B75400575B2
:102BE7005A03755BD69000E2E01475F00584FF7E0A
:102BF70000E538BE00039F5005121188800BE538A9
:102C0700900467127310E0F538E5389008F6F090F5
:102C170008F6E0FE9000D1E0C39E50089000D1E096
:102C27009008F6F09000C0E0D3941D401E9008F67F
:102C3700E0FE90008EE02EFE90005EE075F01E84B0
:102C4700FC7F00EE2C9008F6F08031A237B3400AE3
:102C570090008EE09008F6F080229008F6E0FE9053
:102C67000090E02EFE90008EE02EFE90005EE07554
:102C7700F01E84FC7F00EE2C9008F6F0229000975F
:102C8700E0B40136E56875F00A84FF7E009005918F
:102C9700120048E0F547E547D394644010E547C381
:102CA700946475F00F84FF7E008F4780037547009B
:102CB7009000B4E02547F54780069000B4E0F5475B
:102CC70022E56875F00A84FF7E009005911200489E
:102CD700E0C394694007E568D3946440559000FECB
:102CE700E0C394035026900893E0FEA3E0FF74042A
:102CF700120039E5601272DF740F8E048F05FF1220
:102D070072CF900891ECF0A3EDF08024900893E047
:102D1700FEA3E0FF7404120039E5621272DF740F3C
:102D27008E048F05FF1272CF900891ECF0A3EDF09F
:102D3700800F900893E0F8A3E0900891C8F0A3C82B
:102D4700F0A204401A900893E0FEA3E0FF74031278
:102D570072DF7401120039900891EEF0A3EFF09042
:102D670000A7E0B40262E56BC3944175F00584FFE8
:102D77007E008F38E56B75F00584ADF07C008D3BE8
:102D8700754005755A06755B14E538C394175005E9
:102D970012118880069006B8E0F538900891E0FE99
:102DA700A3E0FF740A8E048F05FF1272CFE5388CFB
:102DB700068D071272DF740A8E048F05FF1272CF19
:102DC700900891ECF0A3EDF0900891E0FEA3E0FFEE
:102DD700900897E0FCA3E0FDEDD39FEC9E400F9099
:102DE7000897E0F8A3E0900891C8F0A3C8F022E59F
:102DF7000875F004A4FFAEF09006D4120048E090E6
:102E07003C4BF8282873804C85537480479000E426
:102E1700E08560F0A4FFAEF074081200398F74806B
:102E270033856274802E856874802985697480244F
:102E3700856A74801F856B74801A856C748015850C
:102E470067748010856674800B856D7480069000AA
:042E57001FE0F5740F
:103C4B00022E0D022E0F022E14022E28022E2D02F2
:103C5B002E32022E37022E3C022E41022E46022E0F
:073C6B004B022E50022E5502
:102E5B00E50875F004A4FFAEF09006D5120048E526
:102E6B000875F004A4FFAEF0E0FC9006D612004803
:102E7B00ECFEE0FFEEC39F4003022F63E50875F005
:102E8B0004A4FFAEF09006D4120048E0B40441E570
:102E9B000875F004A4FFAEF09006D6120048E0C30C
:102EAB009574500AE508F50CD39239123E22E508C9
:102EBB0075F004A4FFAEF09006D5120048E0D39550
:102ECB0074400AE508F50CC39239123E22022F61B9
:102EDB00E50875F004A4FFAEF09006D5120048E0AB
:102EEB00C395745015E50875F004A4FFAEF0900679
:102EFB00D6120048E0D395745002800AE508F50C11
:102F0B00D39239123E22E50875F004A4FFAEF0907F
:102F1B0006D5120048E0D395745015E50875F004FA
:102F2B00A4FFAEF09006D6120048E0C39574500A89
:102F3B00E508F50CC39239123E229006DCE0B40191
:102F4B00099000F0E0D395625002800A7402F50CF0
:102F5B00C39239123E22806AE50875F004A4FFAED5
:102F6B00F09006D5120048E0D395744015E508752E
:102F7B00F004A4FFAEF09006D6120048E0C395749F
:102F8B004002800AE508F50CC39239123E22E5088F
:102F9B0075F004A4FFAEF09006D5120048E0C3957F
:102FAB00744015E50875F004A4FFAEF09006D61238
:102FBB000048E0D39574400AE508F50CD39239121A
:102FCB003E2222AE2FAF3074C9BE000CD39F4008F7
:102FDB00782F1273320230E8753001752F00AE5224
:102FEB00AF53E547BE000DD39F40099000C6E0D319
:102FFB00954840028023754800E547C39553F57407
:10300B009000C9E0D395464008E5462574F5468007
:10301B00069000C9E0F546800205489000A2E0D377
:10302B009562401CE560C395614015AE52AF53E508
:10303B0047BE00039F50099000C7E0D3954940025B
:10304B00806E9008F8E0A852B800049553500375B1
:10305B004B009008F8E0A852B8000BD395534006EC
:10306B00E5539008F8F0E54B7041E553C39547F5F0
:10307B0074E574D3940540037574059000C8E0C3E0
:10308B0095465007E574C3954640028009E546C353
:10309B009574F54680069000C8E0F5469000C8E0B0
:1030AB00D3954640069000C8E0F54675490080026E
:1030BB000549E54B70169000A2E0C39562500DE5F3
:1030CB00472405A852B8000695534002800F900084
:1030DB00B5E0F546754B0174789008F8F022AE2FE9
:1030EB00AF3074E9D39F74039E4008782F1273326C
:1030FB0002328F753001752F00754632A22B402A94
:10310B007546199000B5E075F002A4FFAEF0E548E6
:10311B00BE0006D39F4002D22B0548754B03747833
:10312B009008F8F0754A00023276AE52AF53E5477D
:10313B006F4E7003023276E547BE000DD39F4009F8
:10314B009000C6E0D395484002800F754800E54BD0
:10315B00C394035003754619800DE547C39553F58A
:10316B0074E5482574F5489000A2E0D39562400EB3
:10317B009008F8E0A852B80007D395534002800C92
:10318B00054A9000B5E0B54A03754B00E54BB40317
:10319B0006A204B3B34002800A054AE54AB43C03D5
:1031AB00754B02E54BB402299008F8E0A852B80021
:1031BB000ED395534009E5539008F8F0754A0090EB
:1031CB0000A2E0C395625009754A0074789008F824
:1031DB00F0E54B705A9000A2E0D39562401CE5607D
:1031EB00C395614015AE52AF53E547BE00039F50E8
:1031FB00099000C7E0D395494002800875490075D6
:10320B00464B8028E553C39547F574E574D3940575
:10321B0040037574059000A2E0D395624008E54920
:10322B002574F5498006E5492406F549754A00E5FC
:10323B004B70169000A2E0C39562500DE547240534
:10324B00A852B80006955340028003754B01E54B1D
:10325B00B40118754619054A9000B5E0B54A0675D4
:10326B004B02754A0074789008F8F0A202B3400341
:10327B00754632E54675F00AA4FFAEF090089DEE58
:10328B00F0A3EFF022E570903C72F8282873023C13
:10329B000B90009AE070030235BA9000D0E0B401B5
:1032AB0002800302345090005CE0655F6009E553D7
:1032BB004552600302344D7E017F00E5BE1272DF82
:1032CB00E5BD2FFF50010E8E5A8F5B9000CEE0B400
:1032DB00461B740E1272DF900081E08E048F05FF87
:1032EB001272CF9008A1ECF0A3EDF0801DAE5AAF97
:1032FB005B74101272DF900081E08E048F05FF1259
:10330B0072CF9008A1ECF0A3EDF0E56C600FE56CCB
:10331B00C394FE50089000F6E06402600280649053
:10332B0000E4E0B40B1F9008A1E0FEA3E0FF74E7FC
:10333B001272DFE56C8E048F05FF1272CF9008A11D
:10334B00ECF0A3EDF09000E4E0D3940B4008900078
:10335B00CCE064046002802B9008A1E0FEA3E0FFA8
:10336B009008A5E0FCA3E0FDEFD39DEE9C400D1271
:10337B00732A9008A1EEF0A3EFF080079008A1E468
:10338B00F0A3F09008A1E0FEA3E0FFEFD39400EED2
:10339B0094014008D238742690005FF0A238B3B382
:1033AB00502C7E057F009000E4E08E048F05FF1209
:1033BB0072CF9008A1E0FEA3E0FFEFC39DEE9C400F
:1033CB000FAC52AD53740FBC0004D39D500280025E
:1033DB00C23890009AE0B402279008A3E0FEA3E065
:1033EB00FF9008A1E0FCA3E0FDEF2DFDEE3CFC748B
:1033FB00018C068D071200399008A1EEF0A3EFF0B7
:10340B009008A1E0FEA3E0FF9008A3E0FCA3E0FD81
:10341B00EDD39FEC9E4004D22E8002B22E9008A1D9
:10342B00E0F8A3E09008A3C8F0A3C8F09000CCE0AC
:10343B0064016006A22EB3B3400280069008A2E09E
:10344B00F5600235B8D22E7E017F00E5BE1272DF29
:10345B00E5BD2FFF50010E8E5A8F5B9000CEE0B46E
:10346B00461B740E1272DF900081E08E048F05FFF5
:10347B001272CF9008A1ECF0A3EDF0801DAE5AAF05
:10348B005B74101272DF900081E08E048F05FF12C7
:10349B0072CF9008A1ECF0A3EDF0E56C600FE56C3A
:1034AB00C394FE50089000F6E064026002806490C2
:1034BB0000E4E0B40B1F9008A1E0FEA3E0FF74E76B
:1034CB001272DFE56C8E048F05FF1272CF9008A18C
:1034DB00ECF0A3EDF09000E4E0D3940B40089000E7
:1034EB00CCE064046002802B9008A1E0FEA3E0FF17
:1034FB009008A5E0FCA3E0FDEFD39DEE9C400D12E0
:10350B00732A9008A1EEF0A3EFF080079008A1E4D6
:10351B00F0A3F09008A1E0FEA3E0FFEFD39400EE40
:10352B0094014008D238742690005FF0A238B3B3F0
:10353B00502C7E057F009000E4E08E048F05FF1277
:10354B0072CF9008A1E0FEA3E0FFEFC39DEE9C407D
:10355B000FAC52AD53740FBC0004D39D50028002CC
:10356B00C23890009AE0B402279008A3E0FEA3E0D3
:10357B00FF9008A1E0FCA3E0FDEF2DFDEE3CFC74F9
:10358B00018C068D071200399008A1EEF0A3EFF025
:10359B009008A1E0F8A3E09008A3C8F0A3C8F090AE
:1035AB0000CCE0640160069008A2E0F56080037532
:1035BB006000900096E0700675700302329075BB48
:1035CB0018023C0B023C0B900096E0700302374351
:1035DB007E017F00E5BE1272DFE5BD2FFF50010EAD
:1035EB008E5A8F5B9000DCE0B4010F7E0F7FFFAC37
:1035FB005AAD5B12732A8E5A8F5B900101E0B402B5
:10360B0045AE5AAF5B900028E0FCA3E0FDEDD39FE5
:10361B00EC9E400A900028E55AF0A3E55BF0AE5A09
:10362B00AF5B90002AE0FCA3E0FDEFD39DEE9C4046
:10363B000A90002AE55AF0A3E55BF0AE5AAF5B7433
:10364B00041200398F62900101E0704CAE5AAF5BEF
:10365B00900028E0FCA3E0FDEFD39DEE9C40091207
:10366B00732A8E5A8F5B8006755B00755A00AE5AB3
:10367B00AF5B74101272DF900100E08E048F05FFB8
:10368B001272CF8C5A8D5B74FFBC0009D39D400521
:10369B00855B6280037562FE9000CCE0B401028012
:1036AB0003023741A204B3B3500E9000A0E0A8521E
:1036BB00B80005D39553500280719000DDE0856210
:1036CB00F0A4FFAEF074648E048F05FF1272CF8CE2
:1036DB005A8D5BE56C6016E56CC394FE500F900041
:1036EB00F6E0B402089000E4E0640B60028017AED1
:1036FB005AAF5B74E71272DFE56C8E048F05FF1215
:10370B0072CF8C5A8D5BAE5AAF5B9008A1E0FCA3D5
:10371B00E0FDEDD39FEC9E4005855B60800BA22EF8
:10372B00B340069008A2E0F560800BA22EB34006D2
:10373B009008A2E0F5608003756200900099E0703C
:10374B000675700502329075BB19023C0B023C0BDF
:10375B00900099E070030237FBE55FD3955E400361
:10376B000237F9900026E0FEA3E0FFE56612732214
:10377B00900026EEF0A3EFF07E017F00E5BE127203
:10378B00DFE5BD2FFF50010E8E5A8F5B900106E0D7
:10379B007013740A1272DF74518E048F05FF12724C
:1037AB00CF8D668019AE5AAF5B740A1272DF8F042D
:1037BB008E057E017F95CDCCCD1271CD8F66E566E2
:1037CB00D394644003756664900026E0FEA3E0FF8B
:1037DB00E5662FFF50010E900026EEF0A3EFF09060
:1037EB00009DE0048E048F05FF1272CF8D6680035F
:1037FB007566329000E9E0700675700702329075BD
:10380B00BB13023C0B023C0B9000E9E0604A7E01CB
:10381B007F00E5BE1272DFE5BD2FFF50010E8E5A01
:10382B008F5B74041200398F679000EBE08567F0B3
:10383B00A4FDACF07464FF1272CF8D679000EAE0C8
:10384B008567F0A4FFAEF074FF8E048F05FF127234
:10385B00CFED900080F08003756700900097E070CB
:10386B000675700902329075BB17023C0B023C0BBC
:10387B00900097E0B40102800302390F7E017F00B4
:10388B00E5BE1272DFE5BD2FFF50010E8E5A8F5B26
:10389B009008F9E060199008F9E014906CEC1200B4
:1038AB008CE493FC740193FDEDC39FEC9E4002806E
:1038BB00069008F9E014F09008F9E0C394B3501D9A
:1038CB00AE5AAF5B9008F9E004906CEC12008CE4FC
:1038DB0093FC740193FDEFC39DEE9C400280069018
:1038EB0008F9E004F09008F9E0FE9000BDE08E00CE
:1038FB0088F0A4FFAEF074648E048F05FF1272CFB4
:10390B008D688003756800900098E0700675700BE9
:10391B0002329075BB16023C0B023C0B900098E0F8
:10392B00B4010280030239BB7E017F00E5BE127237
:10393B00DFE5BD2FFF50010E8E5A8F5B9008FAE02A
:10394B0060199008FAE014906E5612008CE493FC08
:10395B00740193FDEDC39FEC9E400280069008FA24
:10396B00E014F09008FAE0C394B3501DAE5AAF5B6D
:10397B009008FAE004906E5612008CE493FC7401EC
:10398B0093FDEFC39DEE9C400280069008FAE00485
:10399B00F09008FAE0FE9000C3E08E0088F0A4FFE0
:1039AB00AEF074648E048F05FF1272CF8D698003A5
:1039BB0075690075BB1F023C0B023C0B7E017F003F
:1039CB00E5BE1272DFE5BD2FFF50010E8E5A8F5BE5
:1039DB0074091272DF74E68E048F05FF1272CF8D9D
:1039EB006B90009FE0700675700F02329075BB15DF
:1039FB00023C0B023C0B90009FE07003023B527E9B
:103A0B00017F00E5BE1272DFE5BD2FFF50010E8E68
:103A1B005A8F5B74041200398F6A90009FE0B401D7
:103A2B00159000F3E0856AF0A4FFAEF07407120066
:103A3B0039EF9008F4F090009FE0B402159000F37A
:103A4B00E0856AF0A4FFAEF07407120039EF90081E
:103A5B00F3F090009FE0B403028003023B3590002B
:103A6B00E0E07052E56AC39419500FD22A9000BF60
:103A7B00E09008F7F09008FCE4F0E56AD39464401A
:103A8B0004A22A4002802D9008FCE004F09008FC70
:103A9B00E0FE900132E0B5060B9008F7E004F090E1
:103AAB0008FCE4F09008F7E064966006900132E0C1
:103ABB007002C22A80639000BFE070349000F3E084
:103ACB00856AF0A4FFAEF074FF8E048F05FF1272AF
:103ADB00CFED9008F7F0AE52AF53741EBE0006D375
:103AEB009F4002D22AE562D394E54002C22A802984
:103AFB00E56AC3940A500DAE52AF53741EBE000458
:103B0B00D39F50028002D22AE562D394E54002C2D1
:103B1B002A9000BFE09008F7F09008F7E0C39405F7
:103B2B00500674059008F7F0C22F90009FE0B40484
:103B3B0014E56AC394195002D22FE56AD39432402C
:103B4B0002C22FC22A8003756A009000F6E070064D
:103B5B0075701102329075BB14023C0B023C0B903A
:103B6B0000F6E07003023BF87E017F00E5BE1272A7
:103B7B00DFE5BD2FFF50010E8E5A8F5B90011BE0CE
:103B8B007025EFD39421EE940E4005756CFF8015D4
:103B9B00AE5AAF5B74101272DF74E38E048F05FFA5
:103BAB001272CF8D6C8027AE5AAF5BEFD39449EE78
:103BBB0094064005756CFF8015AE5AAF5B741012FE
:103BCB0072DF74638E048F05FF1272CF8D6CE56C00
:103BDB0075F00BA4FFAEF09000E4E08E048F05FFB0
:103BEB001272CF9008A5ECF0A3EDF08003756C007A
:103BFB0090009AE0600575BB1A800375BB188000B6
:103C720002329902329C0235CF0235D20237580203
:103C8200375B02381002381302387802387B023967
:103C9200240239270239C40239C70239FE023A0125
:093CA200023B67023B6A023C0B85
:103C0B00E57075F00284AFF07E00EF4E7002D2ECDF
:033C1B000570220F
:097310002582F58250020583225A
:0F008C0025E050020583258250020583F582226C
:1072AE00EF2F500205832582F582E5833E2EF5836E
:0172BE0022AD
:10732200CFC39FFF50011E22C3EF9DFFEE9CFE22A2
:087332000806B600021806224D
:0D72ED00A3E004F07006127306E004F02226
:08733A000816B6FF0218162226
:0E003900048007C3CE13CECF13CFD5E0F6223E
:1071CD00BC000FBE0008ED8FF084FFADF022E4FE91
:1071DD00FF22BE000DEF60FE54F0606F20E703024A
:1071ED007283EAC0E0EBC0E078017A0075F001EE41
:1071FD0020E710EF25E0FFEE33FE0AC5F023C5F0C2
:10720D0030E7F0EA5407F9096A7A007B006001085B
:10721D00C3EC9E40167004ED9F4010ED9FFDEC9E5B
:10722D00FCE5F0CA4ACA03F5F08005E5F003F5F078
:10723D00C3EE13FEEF13FFD9D77908CACBCAD8D046
:10724D00EAFEEBFFD0E0FBD0E0FA22EC8FF084FCFD
:10725D00ED54F045F0C48FF084FEEDC454F045F0CC
:10726D00C48FF084FDEEC4FE54F02DFFEE540F3CA0
:10727D00FEADF07C0022790078008FF0EC7E0820C6
:10728D00E70DC3CD33CD33C933C9C833C8DEF08460
:10729D0049F9E5F08FF0BE00E6FD7C00E9FFE8FE60
:0172AD0022BE
:0E72DF00F88FF0A4FFE5F0CE88F0A42EFE227A
:10000300EF8DF0A4F9A8F0EF8CF0A428F8EE8DF0B2
:06001300A428FEE9FF2213
:1072BF00600D782B0272C9007830D8FED5E0F82225
:1072CF00EEC0E07E001271CDEFFDEEFCD0E0FE22AD
:0C72FA00EEC0E07E001271CDD0E0FE225C
:03001B0002001EC2
:0300530002005652
:03009B00020071EF
:030000000273196F
:0973190075817675D000024C1E4E
:0B004800E5822FF582E5833EF5832260
:0A7306000582D5820215831582224C
:10001E00C0E0C0F0C083C082C0D075D000124B8843
:0B002E00D0D0D082D083D0F0D0E032E0
:10005600C0E0C0F0C083C082C0D075D000124B8B08
:10006600D0D0D082D083D0F0D0E032C0E0C0F0C093
:1000760083C082C0D075D000124BE0D0D0D082D0E1
:0600860083D0F0D0E0324F
:00000001FF
